:020000040800F2
:10000000008000209D7F00082D1700082F17000892
:1000100031170008331700083517000800000000EA
:10002000000000000000000000000000371700087A
:1000300039170008000000003B1700083D170008B2
:10004000ED7F0008ED7F0008ED7F0008ED7F0008E0
:10005000ED7F0008ED7F0008ED7F0008ED7F0008D0
:10006000ED7F0008ED7F0008ED7F0008ED7F0008C0
:10007000ED7F0008ED7F0008ED7F0008ED7F0008B0
:10008000ED7F000800000000ED7F0008ED7F000814
:1000900045170008ED7F0008ED7F0008ED7F0008A0
:1000A000ED7F0008ED7F0008ED7F0008ED7F000880
:1000B000ED7F000855170008ED7F0008ED7F000870
:1000C000ED7F0008ED7F0008ED7F0008ED7F000860
:1000D000ED7F0008ED7F0008ED7F0008ED7F000850
:1000E000ED7F0008ED7F0008ED7F0008ED7F000840
:1000F000ED7F0008ED7F0008ED7F000800000000A4
:1001000000000000ED7F000800000000ED7F000807
:10011000ED7F000800000000ED7F0008ED7F000883
:10012000ED7F0008ED7F0008ED7F0008ED7F0008FF
:10013000ED7F00080000000000000000ED7F0008D7
:10014000ED7F0008ED7F00080000000000000000C7
:10015000000000000000000000000000000000009F
:10016000000000000000000000000000ED7F00081B
:10017000ED7F00080000000000000000000000000B
:1001800000000000ED7F00080000000000000000FB
:10019000000000000000000000000000000000005F
:1001A0000000000000000000ED7F0008ED7F000867
:1001B000ED7F0008ED7F0008ED7F000800000000E3
:1001C00000000000ED7F00080000000000000000BB
:0801D000ED7F0008ED7F00083F
:1001D8000348044B834202D0034B03B118477047CE
:1001E8003001002030010020000000000548064BC7
:1001F8001B1AD90F01EBA301491002D0034B03B11D
:10020800184770473001002030010020000000002E
:1002180010B5064C237843B9FFF7DAFF044B13B146
:100228000448AFF300800123237010BD3001002083
:1002380000000000F07F000808B5044B1BB104491A
:100248000448AFF30080BDE80840CFE70000000095
:1002580034010020F07F000870B50D4E0D4D761B5F
:10026800B61006D0002455F8043B01349847A6423E
:10027800F9D1094E094D761B07F0B6FEB61006D027
:10028800002455F8043B01349847A642F9D170BDC3
:1002980098800008988000089C80000898800008D2
:1002A800830730B548D0541E002A3FD0CAB203464F
:1002B80001E0013C3AD303F8012B9D07F9D1032C47
:1002C8002DD9CDB245EA05250F2C45EA054536D985
:1002D800A4F1100222F00F0C03F1200EE6444FEABD
:1002E800121C03F1100242E9045542E9025510328A
:1002F8007245F8D10CF1010214F00C0F03EB021255
:1003080004F00F0C13D0ACF1040323F003030433FF
:10031800134442F8045B9342FBD10CF003042CB164
:10032800CAB21C4403F8012B9C42FBD130BD644681
:100338001346002CF4D1F9E703461446BFE71A46E2
:10034800A446E0E781F0004102E000BF83F00043EB
:1003580030B54FEA41044FEA430594EA050F08BF58
:1003680090EA020F1FBF54EA000C55EA020C7FEA1C
:10037800645C7FEA655C00F0E2804FEA5454D4EB99
:100388005555B8BF6D420CDD2C4480EA020281EA63
:10039800030382EA000083EA010180EA020281EA9B
:1003A8000303362D88BF30BD11F0004F4FEA0131ED
:1003B8004FF4801C4CEA113102D0404261EB4101FC
:1003C80013F0004F4FEA03334CEA133302D0524282
:1003D80063EB430394EA050F00F0A780A4F101043E
:1003E800D5F1200E0DDB02FA0EFC22FA05F2801878
:1003F80041F1000103FA0EF2801843FA05F359415E
:100408000EE0A5F120050EF1200E012A03FA0EFCDC
:1004180028BF4CF0020C43FA05F3C01851EBE37106
:1004280001F0004507D54FF0000EDCF1000C7EEB23
:1004380000006EEB0101B1F5801F1BD3B1F5001F61
:100448000CD349085FEA30004FEA3C0C04F1010480
:100458004FEA445212F5800F80F09A80BCF1004FA9
:1004680008BF5FEA500C50F1000041EB045141EA2B
:10047800050130BD5FEA4C0C404141EB0101013CF4
:1004880028BFB1F5801FE9D291F0000F04BF0146E3
:100498000020B1FA81F308BF2033A3F10B03B3F1B5
:1004A80020020CDA0C3208DD02F1140CC2F10C0245
:1004B80001FA0CF021FA02F10CE002F11402D8BFA3
:1004C800C2F1200C01FA02F120FA0CFCDCBF41EA6F
:1004D8000C019040E41AA2BF01EB0451294330BD3E
:1004E8006FEA04041F3C1CDA0C340EDC04F114041B
:1004F800C4F1200220FA04F001FA02F340EA0300F2
:1005080021FA04F345EA030130BDC4F10C04C4F137
:10051800200220FA02F001FA04F340EA0300294617
:1005280030BD21FA04F0294630BD94F0000F83F461
:10053800801306BF81F480110134013D4EE77FEA44
:10054800645C18BF7FEA655C29D094EA050F08BF90
:1005580090EA020F05D054EA000C04BF1946104671
:1005680030BD91EA030F1EBF0021002030BD5FEAB5
:10057800545C05D14000494128BF41F0004130BDDD
:1005880014F580043CBF01F5801130BD01F0004531
:1005980045F0FE4141F470014FF0000030BD7FEAA4
:1005A800645C1ABF194610467FEA655C1CBF0B469F
:1005B800024650EA013406BF52EA033591EA030FB6
:1005C80041F4002130BD00BF90F0000F04BF0021AE
:1005D800704730B54FF4806404F132044FF00005E1
:1005E8004FF0000150E700BF90F0000F04BF00215A
:1005F800704730B54FF4806404F1320410F00045C0
:1006080048BF40424FF000013EE700BF42004FEABA
:10061800E2014FEA31014FEA02701FBF12F07F4337
:1006280093F07F4F81F06051704732F07F4208BFEE
:10063800704793F07F4F04BF41F40021704730B5F5
:100648004FF4607401F0004521F000411CE700BF41
:1006580050EA010208BF704730B54FF000050AE0C4
:1006680050EA010208BF704730B511F0004502D5C5
:10067800404261EB41014FF4806404F132045FEAC7
:10068800915C3FF4D8AE4FF003025FEADC0C18BF70
:1006980003325FEADC0C18BF033202EBDC02C2F162
:1006A800200300FA03FC20FA02F001FA03FE40EAF4
:1006B8000E0021FA02F11444BDE600BF70B54FF0F8
:1006C800FF0C4CF4E06C1CEA11541DBF1CEA1355D6
:1006D80094EA0C0F95EA0C0F00F0DEF82C4481EA3E
:1006E800030621EA4C5123EA4C5350EA013518BF5E
:1006F80052EA033541F4801143F4801338D0A0FB4B
:1007080002CE4FF00005E1FB02E506F00042E0FBF7
:1007180003E54FF00006E1FB03569CF0000F18BFFD
:100728004EF0010EA4F1FF04B6F5007F64F54074A5
:1007380004D25FEA4E0E6D4146EB060642EAC62138
:1007480041EA55514FEAC52040EA5E504FEACE2EA5
:10075800B4F1FD0C88BFBCF5E06F1ED8BEF1004FA8
:1007680008BF5FEA500E50F1000041EB045170BD24
:1007780006F0004646EA010140EA020081EA030168
:10078800B4EB5C04C2BFD4EB0C0541EA045170BD64
:1007980041F480114FF0000E013C00F3AB8014F1DE
:1007A800360FDEBF002001F0004170BDC4F1000427
:1007B800203C35DA0C341BDC04F11404C4F12005A8
:1007C80000FA05F320FA04F001FA05F240EA020003
:1007D80001F0004221F0004110EBD37021FA04F639
:1007E80042EB06015EEA430E08BF20EAD37070BDF3
:1007F800C4F10C04C4F1200500FA04F320FA05F052
:1008080001FA04F240EA020001F0004110EBD37053
:1008180041F100015EEA430E08BF20EAD37070BDC3
:10082800C4F1200500FA05F24EEA020E20FA04F39C
:1008380001FA05F243EA020321FA04F001F000414B
:1008480021FA04F220EA020000EBD3705EEA430EBC
:1008580008BF20EAD37070BD94F0000F0FD101F0EB
:100868000046400041EB010111F4801F08BF013C24
:10087800F7D041EA060195F0000F18BF704703F062
:100888000046520043EB030313F4801F08BF013DE9
:10089800F7D043EA0603704794EA0C0F0CEA1355A5
:1008A80018BF95EA0C0F0CD050EA410618BF52EA5F
:1008B8004306D1D181EA030101F000414FF0000065
:1008C80070BD50EA410606BF1046194652EA430673
:1008D80019D094EA0C0F02D150EA013613D195EAE7
:1008E8000C0F05D152EA03361CBF104619460AD12F
:1008F80081EA030101F0004141F0FE4141F4700139
:100908004FF0000070BD41F0FE4141F4780170BD28
:1009180070B54FF0FF0C4CF4E06C1CEA11541DBF8D
:100928001CEA135594EA0C0F95EA0C0F00F0A7F88F
:10093800A4EB050481EA030E52EA03354FEA0131BC
:1009480000F088804FEA03334FF0805545EA1313CF
:1009580043EA12634FEA022245EA111545EA106597
:100968004FEA00260EF000419D4208BF964244F12E
:10097800FD0404F5407402D25B084FEA3202B61A4D
:1009880065EB03055B084FEA32024FF480104FF421
:10099800002CB6EB020E75EB030E22BFB61A754695
:1009A80040EA0C005B084FEA3202B6EB020E75EB28
:1009B800030E22BFB61A754640EA5C005B084FEA90
:1009C8003202B6EB020E75EB030E22BFB61A75465D
:1009D80040EA9C005B084FEA3202B6EB020E75EB68
:1009E800030E22BFB61A754640EADC0055EA060E29
:1009F80018D04FEA051545EA16754FEA06164FEA6C
:100A0800C30343EA52734FEAC2025FEA1C1CC0D117
:100A180011F4801F0BD141EA00014FF000004FF0A4
:100A2800004CB6E711F4801F04BF01430020B4F165
:100A3800FD0C88BFBCF5E06F3FF6AFAEB5EB030C1D
:100A480004BFB6EB020C5FEA500C50F1000041EB1A
:100A5800045170BD0EF0004E4EEA113114EB5C04E7
:100A6800C2BFD4EB0C0541EA045170BD41F48011BA
:100A78004FF0000E013C90E645EA060E8DE60CEAC2
:100A8800135594EA0C0F08BF95EA0C0F3FF43BAFDF
:100A980094EA0C0F0AD150EA01347FF434AF95EA96
:100AA8000C0F7FF425AF104619462CE795EA0C0F7A
:100AB80006D152EA03353FF4FDAE1046194622E747
:100AC80050EA410618BF52EA43067FF4C5AE50EA21
:100AD80041047FF40DAF52EA43057FF4EBAE12E711
:100AE8004FEA410212F5001215D211D56FF478734E
:100AF800B3EB625212D94FEAC12343F0004343EAF1
:100B0800505311F0004F23FA02F018BF40427047CB
:100B18004FF00000704750EA013005D111F0004055
:100B280008BF6FF0004070474FF00000704700BFEB
:100B38004A0011D212F5001211D20DD56FF4787354
:100B4800B3EB62520ED44FEAC12343F0004343EAA9
:100B5800505323FA02F070474FF00000704750EAF4
:100B6800013002D14FF0FF3070474FF0000070475E
:100B780053B94AB9002908BF00281CBF4FF0FF31FC
:100B88004FF0FF3000F06AB9ADF1080C6DE904CE02
:100B980000F006F8DDF804E0DDE9022304B0704750
:100BA8002DE9F047089D0C46002B4ED194468C4504
:100BB8008646B2FA82F262D94AB1C2F12003914064
:100BC80020FA03F30CFA02FC194300FA02FE4FEA7A
:100BD8001C471FFA8CF6B1FBF7F44FEA1E4307FBDC
:100BE800141143EA014304FB06F199420AD91CEBAC
:100BF800030304F1FF3080F01381994240F2108121
:100C0800023C6344591A1FFA8EF3B1FBF7F007FB55
:100C1800101143EA014300FB06F69E420AD91CEB79
:100C2800030300F1FF3180F0FD809E4240F2FA801C
:100C3800634402389B1B40EA044000211DB1D340A5
:100C48000022C5E90032BDE8F0878B4205D90DB115
:100C5800C5E9000100210846F5E7B3FA83F1002948
:100C680046D1A34202D39042C0F0F180861A64EBC9
:100C780003030120002DE6D0C5E90063E3E7002A5D
:100C880040F09180A1EB0C044FEA1C481FFA8CF746
:100C98000121B4FBF8F64FEA1E4308FB164443EA69
:100CA800044307FB06F0984208D91CEB030306F13E
:100CB800FF3402D2984200F2CE8026461C1A1FFA50
:100CC8008EF3B4FBF8F008FB104443EA044300FB3E
:100CD80007F79F4208D91CEB030300F1FF3402D247
:100CE8009F4200F2B1802046DB1B40EA0640A5E7A0
:100CF800C1F120068B4022FA06F71F4320FA06FCB2
:100D080004FA01F343EA0C03F44000FA01F8380C42
:100D18004FEA1349B4FBF0FE1FFA87FC00FB1E44A0
:100D280049EA04440EFB0CF9A14502FA01F20AD97A
:100D38003C190EF1FF3A80F08580A14540F282808F
:100D4800AEF1020E3C44A4EB09041FFA83F9B4FB8C
:100D5800F0F300FB134449EA044403FB0CFCA445EC
:100D680007D93C1903F1FF3068D2A44566D9023B84
:100D78003C4443EA0E40A0FB0293A4EB0C049C42C3
:100D8800CE469C4652D34FD055B1B8EB0E0364EB18
:100D98000C0404FA06F6CB40CC401E43C5E90064B7
:100DA8000021BDE8F087C2F1200320FA03F10CFA14
:100DB80002FC24FA03F394400C434FEA1C4800FA5F
:100DC80002FE1FFA8CF7B3FBF8F008FB1031230C76
:100DD80043EA014300FB07F1994208D91CEB0303DE
:100DE80000F1FF362CD299422AD9023863445B1AA3
:100DF800A4B2B3FBF8F108FB113344EA034401FB46
:100E080007F3A34208D91CEB040401F1FF3613D2FF
:100E1800A34211D902396444E41A41EA004138E78F
:100E28000446EFE6084605E7C845ADD2B9EB020E21
:100E380063EB070C0138A7E73146EDE7034698E76F
:100E48003046D4E7D6467EE7634402384CE7064688
:100E5800234608460EE7023E63442FE7704700BF6B
:100E680000B58BB000230593069307930893099365
:100E780003F1804303F50433DA6C42F02002DA64AC
:100E8800DA6C02F020020192019ADA6C42F0400218
:100E9800DA64DA6C02F040020292029ADA6C42F0EA
:100EA8000102DA64DA6C02F001020392039ADA6C46
:100EB80042F00202DA64DB6C03F002030493049B41
:100EC8004FF4806305930223069305A9024801F0B5
:100ED800E3FB0BB05DF804FB0018004872B6FEE7B0
:100EE80000B58FB000230A930B930C930D930793CF
:100EF8000893099300930193029303930493059332
:100F0800069332484FF0804202604360836040F2AB
:100F1800FF72C2600361836103F0BEF9002844D107
:100F28004FF480530A930AA9284803F005FB0028C8
:100F38003DD1264803F0E0F900283AD10023079371
:100F4800099307A9214803F053FC002833D16023F3
:100F580000934FF4FA7301930022029204926946B7
:100F68001A4803F03FFA40BB4FF47A730193042206
:100F78006946164803F036FA08BB40F2DC53019381
:100F880008226946114803F02DFAD0B94FF4FA63E4
:100F980001930C2269460D4803F024FA98B90B48CE
:100FA80000F008FD0FB05DF804FBFFF797FFFFF7AF
:100FB80095FFFFF793FFFFF791FFFFF78FFFFFF70D
:100FC8008DFFFFF78BFFFFF789FF00BF2802002086
:100FD80008B51148114B0360114B4360002383602F
:100FE8000122C260036143618361C361036202F04D
:100FF8000FFB50B90021084802F0CAFD38B900219A
:10100800054802F0F3FD20B908BDFFF767FFFFF7B9
:1010180065FFFFF763FF00BF740200200054004023
:10102800C180802000B589B00023049305930693FE
:1010380007930193029303931348144A02604FF4F1
:10104800404242608360C722C2600361836103F04B
:1010580023F990B94FF48053049304A90A4803F084
:101068006BFA60B900230193039301A9064803F0C2
:10107800BFFB30B909B05DF804FBFFF72FFFFFF79E
:101088002DFFFFF72BFF00BFDC010020000400400C
:1010980010B58CB0002409940A940B9420222146A0
:1010A80001A8FFF7FDF81E484FF0A04303604FF476
:1010B800003343608460C460046144610423836135
:1010C800047744770123036280F82440C4620463F0
:1010D80080F83840C46380F8404001F0FFFCC8B98C
:1010E8000023099309A90E4802F04AF8A0B90D4B4C
:1010F800019306230293002303937F220492042280
:10110800059206930DEB0201054801F007FE28B988
:101118000CB010BDFFF7E2FEFFF7E0FEFFF7DEFEC2
:101128002C0300200080F03E00B589B02022002169
:101138006846FFF7B5F82848284B03604FF400339A
:10114800436000238360C360036101224261082277
:101158008261037743770422026280F82430C362F5
:10116800036380F83830C36380F8403001F0B6FC80
:1011780038BB1B4B009306230193002302937F2265
:1011880003920422049205936946134801F0C6FDB0
:10119800C8B90C23019369460F4801F0BFFDA0B9F7
:1011A8001223019369460C4801F0B8FD78B9182359
:1011B80001936946084801F0B1FD50B909B05DF8DE
:1011C80004FBFFF78BFEFFF789FEFFF787FEFFF7AB
:1011D80085FEFFF783FE00BFC0020020000100501B
:1011E8000800900C08B51548154B03604FF4E1331F
:1011F800436000238360C36003610C224261836102
:10120800C36103624362836203F0F1FD70B9002198
:101218000A4803F064FE58B90021084803F084FE28
:1012280040B9064803F03CFE30B908BDFFF756FE4A
:10123800FFF754FEFFF752FEFFF750FE4C01002067
:101248000038014000B595B03822002106A8FFF704
:1012580027F80023019302930393049305934FF413
:10126800007001F003FB212306934FF480330793AA
:1012780001230C9302230D9303220E920F93202235
:101288001092119304221292139306A800F086FC80
:10129800A0B90F2301930321029100230393049320
:1012A800059301A800F060FF50B900224FF080615B
:1012B800044800F0E7FE15B05DF804FBFFF70EFEEA
:1012C800FFF70CFE0004060008B500F005FCFFF768
:1012D800B9FFFFF7C5FDFFF703FEFFF779FEFFF73C
:1012E800A1FEFFF7D5FEFFF71FFFFFF77BFF03F017
:1012F8004BFE1D4C204602F01BFE1C4802F018FE57
:101308000021204603F0C4F90421204603F0C0F967
:101318000821204603F0BCF90C21204603F0B8F957
:101328000A2000F0FBFB00F03DF90A2000F0F6FB74
:10133800002000F0E9F9012000F0E6F90C4C00214A
:10134800204600F095F90121204600F091F90A2085
:1013580000F0E4FB064C0021204600F089F9012149
:10136800204600F085F9F2E728020020DC01002081
:1013780040420F0010B586B004468DF8171064235C
:101388000322C021094802F04DFB0028F7D164234D
:101398000293012301930DF1170200922246C02106
:1013A800024802F093F906B010BD00BF7402002095
:1013B80010B586B00446059164230322C02109486C
:1013C80002F030FB0028F7D1642302930123019334
:1013D80005AA00922246C021024802F04BFA06B044
:1013E80010BD00BF740200202DE9F84F80460C465E
:1013F800674B984249D8674B984238D9FFF7E4F8C9
:1014080002460B465CA1D1E90001FFF781FAFFF71C
:101418008FFB05282ED910F0010F2CD001302AE0BF
:10142800760001357F2E04DC08FB06F2594B9A4200
:10143800F6D92D01374608FB06F0FFF7C5F8024636
:101448000B464DA1D1E90001FFF762FAFFF770FBE7
:1014580010F0010F00D0013000FB07F708FB07F779
:101468004D4B9F424ED802304FF0000A12E0002543
:101478000126D7E7062008FB00F2474B9A4244D8DA
:10148800023001260025AA4604E0012600254FF077
:101498000C0A042000F10077043FFF0106FB00F06E
:1014A80008FB00F0FFF790F835A3D3E90023FFF716
:1014B8002FFA80468946FFF713FB0646FFF794F894
:1014C80002460B4640464946FEF740FF804689469D
:1014D8002DA3D3E90023FFF7F1F8FFF729FB834693
:1014E800B8B1FFF771F842464B46FFF711FA0022F0
:1014F8002A4BFEF72DFFFFF71BFBB0F5801F09D322
:10150800274807E04FF0000AC4E701260025AA464D
:10151800C0E723484FEACB1BBBFBF0F303EBC6162F
:10152800A6F5007600FB13BB030A23706070C6F3B0
:101538000143A370330AE3702671000B00F0F0003A
:10154800CBF30343184360714FEA1B23A37184F85C
:1015580007B000232372012262725544EDB2C7F32B
:1015680001421544A5723A0AE27227736373A373A2
:10157800E373BDE8F88F00BF00000000A3E1C1419C
:101588000000000060E3764100000000FEFF2F41EC
:1015980080D1F00868780400FF45C3230000E03FCD
:1015A800FFFF0F0010B5002421460020FFF700FFC1
:1015B80010F0800FF8D1FF212C4B19700320FFF792
:1015C800D9FE00210F20FFF7D5FE00211820FFF7D4
:1015D800D1FE00212A20FFF7CDFE01212B20FFF7A5
:1015E800C9FE00212F20FFF7C5FE00213020FFF79C
:1015F800C1FE00213120FFF7BDFE00213220FFF798
:10160800B9FE01213320FFF7B5FE00213720FFF78F
:10161800B1FE00213820FFF7ADFE00213920FFF789
:10162800A9FE00213A20FFF7A5FE01213B20FFF784
:10163800A1FE00213F20FFF79DFE00214020FFF77B
:1016480099FE00214120FFF795FE4F211020FFF75A
:1016580091FE5F211120FFF78DFE6F211220FFF709
:1016680089FE1221B720FFF785FE10BD98030020E0
:1016780010B584B00C466946FFF7B6FE94B1012C4C
:101688001FD100242EE004F110036B4404F11A006A
:1016980013F8101CC0B2FFF76DFE0134072CF2DD01
:1016A8000A240CE00024F9E704F110036B4404F168
:1016B800220013F8101CC0B2FFF75CFE01340C2C9A
:1016C800F2DD2021B120FFF755FE04B010BD04F172
:1016D80010036B4404F1220013F8101CC0B2FFF78A
:1016E80049FE0134072CF2DD0A240AE004F1100354
:1016F8006B4404F12A0013F8101CC0B2FFF73AFE3D
:1017080001340C2CF2DDDCE708B501238340044AE0
:10171800117821EA030111700320FFF72BFE08BDA1
:1017280098030020FEE7FEE7FEE7FEE7FEE77047C6
:101738007047704708B500F0DFF908BD08B50248E2
:1017480004F008FC08BD00BF4822002008B5024884
:1017580002F036FC08BD00BFDC01002000B583B0F4
:101768000B4B1A6E42F001021A661A6E02F0010261
:101778000092009A9A6D42F080529A659B6D03F030
:1017880080530193019B01F0F7F803B05DF804FB67
:101798000010024010B59AB0044600211591169128
:1017A800179118911991442204A8FEF779FD23682E
:1017B800B3F1A04F04D0364A934234D01AB010BDCA
:1017C8004FF4004304934FF00053139304A800F020
:1017D800F1FDD0B92F4A136801331360012B17D0DC
:1017E8002D4BDA6C42F00202DA64DB6C03F0020380
:1017F8000193019B01231593032316930023179349
:1018080015A9264800F048FFD8E7FFF767FBE1E78E
:10181800214BDA6C42F40052DA64DB6C03F40053B7
:101828000093009BDCE74FF4004304934FF0005310
:10183800139304A800F0BEFDD8B9164A1368013303
:101848001360012B18D0144BDA6C42F00102DA64F1
:10185800DB6C03F001030393039BF023159303232D
:1018680016930023179315A94FF0904000F014FF2A
:10187800A4E7FFF733FBE0E7074BDA6C42F40052CA
:10188800DA64DB6C03F400530293029BDBE700BFCE
:10189800000100509C030020001002400004004892
:1018A800F0B59BB004460021159116911791189137
:1018B8001991442204A8FEF7F3FC2268224B9A42AD
:1018C80001D01BB0F0BD4023049304A800F072FDC2
:1018D800002835D11D4CE36C43F00103E364E36C4D
:1018E80003F001030193019BE36C43F00203E364FB
:1018F800E36C03F002030293029B4FF40043159339
:10190800122716970025179518950426199615A9D4
:101918004FF0904000F0C0FE80231593169717955E
:101928001895199615A90A4800F0B6FEA36D43F458
:101938000013A365A36D03F400130393039BC0E78F
:10194800FFF7CCFAC6E700BF005400400010024081
:101958000004004800B583B00368B3F1804F05D098
:10196800124A93420ED003B05DF804FB03F504332A
:101978009A6D42F001029A659B6D03F00103009392
:10198800009BF0E70A4B9A6D42F002029A659B6D44
:1019980003F002030193019B002211461D2001F070
:1019A80047F81D2001F054F8DDE700BF00040040AF
:1019B8000010024000B587B00023019302930393FF
:1019C800049305930368B3F1804F02D007B05DF824
:1019D80004FB03F50433DA6C42F00102DA64DB6CD1
:1019E80003F001030093009B0F230193022302934A
:1019F8000123059301A94FF0904000F04DFEE5E763
:101A080010B598B0044600211391149115911691C0
:101A18001791442202A8FEF743FC2268184B9A4209
:101A280001D018B010BD0123029302A800F0C2FC37
:101A380010BB144B1A6E42F480421A661A6E02F4F6
:101A480080420092009ADA6C42F00102DA64DB6CA0
:101A580003F001030193019B4FF4C0631393022326
:101A680014930023159316930723179313A94FF084
:101A7800904000F011FED4E7FFF730FAD9E700BF35
:101A88000038014000100240104B1B680BB90120C0
:101A9800704710B504464FF47A70B0FBF3F30C4A64
:101AA8001068B0FBF3F000F0D7FF68B90F2C01D92C
:101AB80001200AE0002221464FF0FF3000F0B8FF75
:101AC800044B1C60002000E0012010BD0000002035
:101AD800080000200400002010B5032000F096FF45
:101AE8000020FFF7D1FF10B10124204610BD0446A5
:101AF800FFF734FEF9E70000034A13680349096851
:101B08000B441360704700BFA003002000000020B2
:101B1800014B1868704700BFA003002038B5044681
:101B2800FFF7F6FF0546B4F1FF3F02D0044B1B68F0
:101B38001C44FFF7EDFF401BA042FAD338BD00BF9D
:101B480000000020124BDA6802F00302DB68C3F3DE
:101B580003130133032A11D00E48B0FBF3F00C4BEA
:101B6800DB68C3F3062303FB00F0094BDB68C3F310
:101B7800416301335B00B0FBF3F070470648B0FBEC
:101B8800F3F0034BDB68C3F3062303FB00F0ECE739
:101B9800001002400024F4000080BB00002800F080
:101BA800548270B582B00446036813F0010F37D031
:101BB800A44A936803F00C03D26802F003020C2BCA
:101BC80023D0082B23D06368B3F5803F4ED0B3F5FC
:101BD800A02F51D09B4B1A6822F480321A601A68E1
:101BE80022F480221A606368002B52D0FFF790FF1E
:101BF8000546944B1B6813F4003F11D1FFF788FF8B
:101C0800401B6428F5D9032028E2032AD9D18D4B3B
:101C18001B6813F4003F03D06368002B00F01782A1
:101C2800236813F0020F5DD0864A936803F00C0313
:101C3800D26802F003020C2B3AD0042B3AD0E368A6
:101C4800002B75D07F4A136843F480731360FFF745
:101C58005FFF05467B4B1B6813F4806F5FD1FFF76E
:101C680057FF401B0228F5D90320F7E1754A13688E
:101C780043F480331360B6E703F18043A3F53C33A4
:101C88001A6842F480221A601A6842F480321A6094
:101C9800A9E7FFF73DFF05466A4B1B6813F4003FB1
:101CA800BED0FFF735FF401B6428F5D90320D5E1E6
:101CB800022AC2D1634B1B6813F4806F03D0E36818
:101CC800002B00F0C6815F4A536823F0FE43216968
:101CD80043EA016353605C4B1868FFF7D5FE0028A0
:101CE80040F0B981236813F0080F4CD063699BB3A7
:101CF800544AD2F8943043F00103C2F89430FFF705
:101D080007FF05464F4BD3F8943013F0020F3AD132
:101D1800FFF7FEFE401B0228F4D903209EE1494A42
:101D2800536823F0FE43216943EA01635360D9E70E
:101D3800444A136823F480731360FFF7E9FE0546ED
:101D4800404B1B6813F4806FCCD0FFF7E1FE401BBB
:101D58000228F5D9032081E13A4AD2F8943023F0D9
:101D68000103C2F89430FFF7D3FE0546354BD3F88C
:101D7800943013F0020F06D0FFF7CAFE401B02286A
:101D8800F4D903206AE1236813F0040F00F081807E
:101D98002C4B9B6D13F0805F36D12A4B9A6D42F025
:101DA80080529A659B6D03F080530193019B012536
:101DB800264B1B6813F4807F28D0A368012B39D0E9
:101DC800052B45D01F4BD3F8902022F00102C3F811
:101DD8009020D3F8902022F00402C3F89020A36842
:101DE800002B43D0FFF794FE0646164BD3F89030ED
:101DF80013F0020F4CD1FFF78BFE801B41F28833A2
:101E08009842F2D9032029E10025D1E70F4A136847
:101E180043F480731360FFF77BFE06460B4B1B6889
:101E280013F4807FC9D1FFF773FE801B0228F5D910
:101E3800032013E1034AD2F8903043F00103C2F8BB
:101E48009030CCE7001002400400002000700040F1
:101E58008A4BD3F8902042F00402C3F89020D3F8BC
:101E6800902042F00102C3F89020B8E7FFF750FE37
:101E78000646824BD3F8903013F0020F08D0FFF7D4
:101E880047FE801B41F288339842F2D90320E5E0EF
:101E9800E5B9236813F0200F35D0A369E3B1774A79
:101EA800D2F8983043F00103C2F89830FFF730FEBB
:101EB8000546724BD3F8983013F0020F23D1FFF781
:101EC80027FE401B0228F4D90320C7E06B4A936D14
:101ED80023F080539365DCE7684AD2F8983023F002
:101EE8000103C2F89830FFF713FE0546634BD3F899
:101EF800983013F0020F06D0FFF70AFE401B0228A5
:101F0800F4D90320AAE0E369002B00F0A6805B4A1D
:101F1800926802F00C020C2A69D0022B1DD0574B94
:101F28001A6822F080721A60DA6822F00302DA6016
:101F3800DA6822F0887222F48032DA60FFF7E8FD6E
:101F480004464E4B1B6813F0007F4ED0FFF7E0FDB0
:101F5800001B0228F5D9032080E0484A136823F0C3
:101F680080731360FFF7D4FD0546444B1B6813F0DC
:101F7800007F06D0FFF7CCFD401B0228F5D90320CF
:101F88006CE03E4AD3683E491940236A606A0138CA
:101F980043EA0013A06A43EA0023206B4008013893
:101FA80043EA4053606B4008013843EA4063E06A03
:101FB80043EAC0631943D160136843F08073136028
:101FC800D36843F08073D360FFF7A2FD04462B4B20
:101FD8001B6813F0007F06D1FFF79AFD001B02284B
:101FE800F5D903203AE0002038E0002036E0012B44
:101FF80036D0224BDB6803F00301226A914231D1CB
:1020080003F0F002616A0139B2EB011F2CD103F42D
:10201800FE42A16AB2EB012F28D103F07842E16AAF
:10202800B2EBC16F24D103F4C001226B5208013A0C
:10203800B1EB425F1ED103F0C063626B5208013AF4
:10204800B3EB426F18D1002008E00120704701204F
:1020580004E0012002E0012000E0002002B070BD91
:102068000120FBE70120F9E70120F7E70120F5E768
:102078000120F3E70120F1E70120EFE7001002401B
:102088000C809F0170B586B00C461546022302935A
:10209800032304930023039300F08056C0F3034CFA
:1020A8000CF5901E0D4AD36C012101FA0CF10B437B
:1020B800D36483B20193C0F30750059001A94FEA96
:1020C8008E2000F0E9FA36B9044A936823F0FE43FB
:1020D8002C431C43946006B070BD00BF0010024042
:1020E8001E4B9B6803F00C03042B33D01B4B9B68DF
:1020F80003F00C03082B2FD0184B9B6803F00C033C
:102108000C2B01D000207047144BDA6802F0030250
:10211800DB68C3F303130133032A11D01048B0FB63
:10212800F3F00E4BDB68C3F3062303FB00F00B4B05
:10213800DB68C3F3416301335B00B0FBF3F0704726
:102148000848B0FBF3F0054BDB68C3F3062303FB39
:1021580000F0ECE702487047024870470010024060
:102168000024F4000080BB00002800F0E680F8B5E9
:102178000C460546744B1B6803F00F038B420BD2C9
:10218800714A136823F00F030B431360136803F0BD
:102198000F038B4240F0D3802E6816F001065FD003
:1021A8006B68032B2FD0022B4DD0684B1B6813F4A0
:1021B800806F00F0C680FFF793FF654B98424DD9BA
:1021C800624A936823F0F00343F08003936080260B
:1021D8005E4A936823F0030369680B439360FFF733
:1021E80097FC0746594B9B6803F00C036A68B3EBEE
:1021F800820F35D0FFF78CFCC01B41F28833984220
:10220800F0D9032078E0514B1B6813F0007F01D10F
:10221800012071E0FFF796FC4D4B98421AD94B4BC1
:102228009B6813F0F00F05D02E6816F00206CFD089
:10223800AB688BB9454A936823F0F00343F08003F9
:1022480093608026C4E7414B1B6813F4003FB2D16A
:10225800012051E00026BBE70026B9E70026B7E7D2
:102268002B6813F0020F48D013F0040F04D0374A3C
:10227800936843F4E06393602B6813F0080F06D06B
:10228800324A936823F47C5343F4E06393602F4A03
:10229800936823F0F003A9680B4393602A4B1B68EB
:1022A80003F00F03A34230D82B6813F0040F06D0B5
:1022B800264A936823F4E063E9680B4393602B682C
:1022C80013F0080F07D0214A936823F46053296953
:1022D80043EAC1039360FFF703FF1C4B9B68C3F3FA
:1022E80003131C4AD35C03F01F03D8401A4B186031
:1022F8001A4B1868FFF7C8FBF8BD802ECED1134AD9
:10230800936823F0F0039360C8E70F4A136823F03B
:102318000F0323431360FFF7FBFB06460A4B1B68BA
:1023280003F00F03A342BFD0FFF7F2FB801B41F27B
:1023380088339842F2D90320DEE701207047012054
:10234800DAE70120D8E700BF002002400010024071
:1023580000B4C404388000080800002004000020ED
:10236800014B1868704700BF0800002008B5FFF748
:10237800F7FF054B9B68C3F30223044AD35C03F0C1
:102388001F03D84008BD00BF00100240308000087D
:1023980008B5FFF7E5FF054B9B68C3F3C223044A62
:1023A800D35C03F01F03D84008BD00BF00100240F3
:1023B80030800008F0B583B00446036813F4002F9A
:1023C80069D0AE4B9B6D13F0805F1ED1AB4B9A6DFD
:1023D80042F080529A659B6D03F080530193019BF4
:1023E8000126A74A136843F480731360FFF790FB34
:1023F8000546A34B1B6813F4807F08D1FFF788FBC1
:10240800401B0228F5D9032502E00026E9E700254C
:1024180045BB9A4BD3F8903013F4407315D0226C17
:102428009A4212D0954AD2F8903023F44073D2F8E9
:10243800901041F48031C2F89010D2F8901021F435
:102448008031C2F89010C2F8903013F0010F10D10B
:1024580045B98A4AD2F8903023F44073216C0B4373
:10246800C2F89030C6B1854A936D23F080539365C6
:1024780012E0FFF74DFB0746804BD3F8903013F07E
:10248800020FE5D1FFF744FBC01B41F288339842A5
:10249800F2D90325DCE70025236813F0010F08D0E3
:1024A800764AD2F8883023F0030361680B43C2F8F8
:1024B8008830236813F0020F08D0704AD2F88830A9
:1024C80023F00C03A1680B43C2F88830236813F08B
:1024D800040F08D0694AD2F8883023F03003E16845
:1024E8000B43C2F88830236813F0080F08D0634AFA
:1024F800D2F8883023F0C00321690B43C2F8883032
:10250800236813F0200F08D05C4AD2F8883023F4EF
:10251800406361690B43C2F88830236813F0400FA9
:1025280008D0564AD2F8883023F44053A1690B43A7
:10253800C2F88830236813F0800F08D04F4AD2F8C9
:10254800883023F44043E1690B43C2F8883023689C
:1025580013F4807F08D0494AD2F8883023F44033F6
:10256800216A0B43C2F88830236813F4007F08D02F
:10257800424AD2F8883023F44023616A0B43C2F8F8
:102588008830236813F4806F0CD03C4AD2F8883026
:1025980023F44013A16A0B43C2F88830A36AB3F549
:1025A800801F57D0236813F4006F0CD0334AD2F839
:1025B800883023F44003E16A0B43C2F88830E36AA9
:1025C800B3F5800F4BD0236813F4805F0CD02B4AEF
:1025D800D2F8883023F04073216B0B43C2F888305F
:1025E800236BB3F1807F3FD0236813F4005F0CD0D6
:1025F800224AD2F8883023F04063616B0B43C2F85B
:102608008830636BB3F1006F33D0236813F4804FC5
:102618000CD01A4AD2F8883023F04063A16B0B43E0
:10262800C2F88830A36BB3F1006F2BD0236813F482
:10263800004F0CD0114AD2F8883023F04053E16B98
:102648000B43C2F88830E36BB3F1805F1FD0284694
:1026580003B0F0BDD36843F48013D360A2E7D36816
:1026680043F48013D360AEE7D36843F48013D36098
:10267800BAE7D36843F48013D360C6E7001002407A
:1026880000700040D36843F48013D360CEE7D3686A
:1026980043F48033D360DAE7F0B583B0002362E017
:1026A80085685E000324B44025EA0405CC68B4407C
:1026B8002C438460456825EA0C054C68C4F3001473
:1026C8009C402C4344605FE0DD08083550F8254005
:1026D80003F0070C4FEA8C0C4FF00F0E0EFA0CFEAD
:1026E80024EA0E0E0C6904FA0CF444EA0E0440F8CD
:1026F800254060E0052400E0002404FA0EF42C4391
:102708000CF1020C554D45F82C40554CA568D443A6
:1027180025EA02064F6817F4801F01D042EA050631
:102728004F4DAE60ED6804EA05064F6817F4001FC8
:1027380001D042EA05064A4DEE606D6804EA0506D6
:102748004F6817F4003F01D042EA0506444D6E6019
:102758002D682C404E6816F4803F01D042EA0504EB
:102768003F4A146001330A6832FA03F474D04FF018
:10277800010C0CFA03FC1CEA0202F3D04C6804F0CA
:102788000304013C012C8BD94C6804F00304032C8E
:102798000CD0C4685D004FF0030C0CFA05FC24EA69
:1027A8000C0C8C68AC4044EA0C04C4604C6804F01F
:1027B8000304022C88D004684FEA430E4FF0030C40
:1027C8000CFA0EFC24EA0C0C4C6804F0030404FA1E
:1027D8000EF444EA0C0404604C6814F4403FC1D081
:1027E800204C256E45F001052566246E04F0010491
:1027F8000194019C4FEA930C0CF10205174C54F814
:10280800255003F0030E4FEA8E0E0F2404FA0EF43F
:1028180025EA0405B0F1904F3FF46EAF124CA04288
:1028280012D004F58064A04210D004F58064A04260
:102838000ED004F58064A0420CD004F58064A04258
:102848003FF458AF062458E7012456E7022454E71A
:10285800032452E7042450E703B0F0BD0000014010
:10286800000401400010024000040048002836D14E
:102878003E4B1B6803F4C063B3F5806F08D03B4A36
:10288800D2F8803023F48073C2F88030002070477B
:10289800364AD2F8803023F48073C2F88030136847
:1028A80023F4C06343F400731360314B1B68322276
:1028B80002FB03F32F4AA2FB03239B0C013300E026
:1028C800013B2A4A526912F4806F01D0002BF7D1DC
:1028D800264B5B6913F4806F44D100207047B0F534
:1028E800007F08D0214A136823F4C06343F480634F
:1028F8001360002070471D4B1B6803F4C063B3F5D9
:10290800806F08D0194AD2F8803043F48073C2F837
:10291800803000207047154AD2F8803043F4807325
:10292800C2F88030136823F4C06343F40073136063
:102938000F4B1B68322202FB03F30E4AA2FB032350
:102948009B0C013300E0013B084A526912F4806F86
:1029580001D0002BF7D1054B5B6913F4806F03D1CD
:102968000020704703207047032070470070004024
:102978000800002083DE1B43024A936843F4804327
:102988009360704700700040002807DB00F01F02CA
:10299800400901239340024A42F82030704700BFA3
:1029A80000E100E0002808DB0901C9B200F160403D
:1029B80000F5614080F80013704700F00F0009012E
:1029C800C9B2014B1954704714ED00E000B500F08E
:1029D8000700C0F1070CBCF1040F28BF4FF0040C2E
:1029E800031D062B0FD9C31E4FF0FF3E0EFA0CF045
:1029F80021EA000199400EFA03FE22EA0E0241EA9A
:102A080002005DF804FB0023EEE70000074AD368E4
:102A180023F4E0631B041B0C000200F4E060034392
:102A280043F0BF6343F40033D360704700ED00E028
:102A380010B50446054BD868C0F30220FFF7C6FF5F
:102A480001462046FFF7AEFF10BD00BF00ED00E0D5
:102A580008B5FFF799FF08BD0138B0F1807F0BD2A8
:102A68004FF0E0235861054AF02182F82310002036
:102A7800986107221A6170470120704700ED00E055
:102A880010B430300B0A9B0003F00C03C45801F05B
:102A98001F014FF01F0C0CFA01FC24EA0C0CC2F3C6
:102AA80084628A404CEA0202C2505DF8044B7047C7
:102AB80010B414304B0E9B0003F00403C458C1F348
:102AC80004514FF0070C0CFA01FC24EA0C0C8A4064
:102AD8004CEA0202C2505DF8044B704730B583B02F
:102AE80000230193002800F00D810446C36D13B341
:102AF80023689A6812F0005F05D09A6822F0204295
:102B080022F03F029A602268936813F0805F1FD119
:102B1800936823F0104323F03F0343F080539360FE
:102B2800794B1B689B09794AA2FB03239B09013354
:102B38005B00019309E0FEF72DFE0023236684F86D
:102B48005830D5E7019B013B0193019B002BF9D13C
:102B58002268936813F0805F40F09C80E36D43F037
:102B68001003E365236E43F0010323660120936895
:102B780013F0040300D00123E16D11F0100F40F0B1
:102B8800BA80002B40F0B780E36D23F4817343F0E3
:102B98000203E365936813F0010F15D14FF0A043CA
:102BA8009A6812F0010200D00122594B9B6813F079
:102BB800010300D00123134306D1636855498A688D
:102BC80022F47C1213438B60627FE36B43EA423347
:102BD800E2681343A268134394F8242043EA0243AB
:102BE800012A59D0E26A22B102F47872216B0A43B1
:102BF80013432168CD68484A2A401A43CA602268AC
:102C0800136923F04063616B0B43136121688B6880
:102C180013F0040300D001238A6812F0080200D0E0
:102C2800012243BB3ABB237F94F83820520042EA82
:102C38008332CB6823F4804323F002031343CB6031
:102C4800236973B32268136943F4803313612268DC
:102C5800D2F8C03023F47F5323F03F0321690B439C
:102C6800C2F8C03094F84030012B29D0226813698B
:102C780023F0010313616369012B33D02268136BBE
:102C880023F00F031363E36D23F0030343F0010301
:102C9800E36535E000206AE7A26A013A43EA424365
:102CA800A0E72268136923F4803313612268D2F8FD
:102CB800C03023F47F5323F03F03C2F8C030D1E77C
:102CC80021680B6923F4FF6323F00403626CA56C8D
:102CD8002A43E56C2A43256D2A43134343F0010335
:102CE8000B61C8E721680B6B23F00F03226A013AD6
:102CF80013430B63C7E7E36D43F01003E36501205B
:102D080003B030BD0120FBE708000020632D3E051D
:102D180000010050000300500740F0FFF0B583B0F9
:102D28000023019390F85830012B00F01E820446CE
:102D38000D46012380F858300068836813F0040FAB
:102D480009D0E36D43F02003E3650120002384F8F4
:102D5800583003B0F0BD0A684968FFF791FE206853
:102D6800836813F0040300D00123866816F0080670
:102D780000D00126002B3ED1002E3CD1AA68B2F12A
:102D8800004F6BD02968FFF793FE2268536923F040
:102D98000043536169692268D368C3F3C1035B00C8
:102DA80099402869042866D0603252F82070A84BF0
:102DB8003B402F6807F0F84C41EA0C010B4343F005
:102DC800004342F8203023682869AA69603353F821
:102DD800201021F080710A4343F8202023682969D4
:102DE8002A7F012A44D0603353F8212022F0007250
:102DF800324343F8212023689A6812F0010F12D158
:102E08002A68E8689349884200F09C80D3F8B0109B
:102E1800C2F3120221EA0202C3F8B020EA688D4B1D
:102E28009A4200F097802B688B4A134200F09581F4
:102E38008A4A926802F0E0718948834200F044812E
:102E48008848834200F040818748834200F06281CD
:102E58008648834200F07081002077E700222968C5
:102E6800FFF726FE2268536943F00043536191E758
:102E78004FF00076B7E7136E116EC1F384612B68CB
:102E8800C3F3120078BBC3F38463994233D021683B
:102E98004B6E4A6EC2F384622B68C3F3120078BB90
:102EA800C3F384639A4233D021688B6E8A6EC2F36F
:102EB80084622B68C3F3120078BBC3F384639A421D
:102EC80033D02168CB6ECA6EC2F384622B68C3F319
:102ED800120078BBC3F384639A428CD1CB6E23F083
:102EE8000043CB6687E793FAA3F313B1B3FA83F3EE
:102EF800CBE72023C9E7136E23F000431366C6E728
:102F080093FAA3F313B1B3FA83F3CBE72023C9E70A
:102F18004B6E23F000434B66C6E793FAA3F313B155
:102F2800B3FA83F3CBE72023C9E78B6E23F0004382
:102F38008B66C6E793FAA3F313B1B3FA83F3CBE72F
:102F48002023C9E7D3F8B010C2F312020A43C3F82A
:102F5800B02063E720682B68C3F3120626BB9A0EDD
:102F6800013202F01F02092A8CBF00220122002A26
:102F780052D046BB990E0131890601F0F84176BB63
:102F88009F0E013707F01F070122BA401143AEBB5D
:102F98009B0E013303F01F0303EB43031B05194387
:102FA800AA68FFF785FD3EE793FAA3F24AB1B2FAA1
:102FB80082F2013202F01F02092A8CBF002201228C
:102FC800D5E72022F5E793FAA3F131B1B1FA81F1FF
:102FD8000131890601F0F841D1E72021F8E793FA99
:102FE800A3F24AB1B2FA82F2013202F01F024FF0A4
:102FF800010C0CFA02F2C9E72022F5E793FAA3F3D1
:1030080043B1B3FA83F3013303F01F0303EB430324
:103018001B05C4E72023F6E756BB990E0131890644
:1030280001F0F84186BB9F0E013707F01F07012208
:10303800BA401143BEBB9B0E013303F01F0303EBE1
:1030480043031E3B1B0543F000731943A8E700BF69
:1030580000F0FF0300007F400000088000030050DC
:10306800000021C31000C090000052C7000084CBAC
:1030780093FAA3F131B1B1FA81F10131890601F076
:10308800F841CFE72021F8E793FAA3F24AB1B2FA60
:1030980082F2013202F01F024FF0010C0CFA02F228
:1030A800C7E72022F5E793FAA3F35BB1B3FA83F3FA
:1030B800013303F01F0303EB43031E3B1B0543F0DF
:1030C8000073C2E72023F3E712F4000F7FF4BCAECD
:1030D8002368B3F1A04F01D0002037E641F4000186
:1030E800234A936823F0E07319439160214B1B68CE
:1030F8009B09214AA2FB03239B09013303EB4303EA
:103108009B000193019B1BB1019B013B0193F9E7D4
:1031180000201BE612F0807F7FF49AAE2268174BDE
:103128009A421CD041F08071114A936823F0E073F1
:1031380019439160002009E612F4800F11D122682A
:103148000E4B9A420FD041F4800309498A6822F055
:10315800E07213438B600020F8E50020F6E50020BC
:10316800F4E50020F2E50020F0E50220F1E500BFDB
:103178000003005008000020632D3E0500010050A8
:1031880090F85820012A7FD010B49DB00346012240
:1031980080F858200022189219920068B0F1A04FC8
:1031A80039D000220192019A002A37D0926812F091
:1031B800040200D00122806810F0040F54D1002AC4
:1031C80052D10A68002A32D0304CA26822F46042F8
:1031D800486893F838C040EA4C300243A2604FF088
:1031E800A042906810F0010000D00120284A92689F
:1031F80012F0010200D00122024341D1234CA268FF
:1032080022F4716222F00F020868896801430A43B8
:10321800A26000202DE01E4A0192C4E7DA6D42F058
:103228002002DA65002283F85820012024E017499B
:103238008A6822F460428A604FF0A042916811F0D7
:10324800010100D00121124A926812F0010200D057
:1032580001220A4316D10D498A6822F4716222F0CC
:103268000F028A60002004E0DA6D42F02002DA657D
:103278000120002283F858201DB05DF8044B7047E8
:103288000020F6E70020F4E7022070470003005012
:103298000001005003689A6912F0020F01D0002261
:1032A8009A6203689A6912F0010F03D19A6942F091
:1032B80001029A61704710B4019CC1F3090141EA07
:1032C80002411943214321F0004102685368640D0B
:1032D80004F4806444F07F7444F4583444F47F74F4
:1032E80044F0030423EA04030B4353605DF8044BE2
:1032F80070472DE9F041044603689F6917F01007ED
:103308004CD00E4690461022DA6100252368986951
:1033180010F0200F3BD1002D39D1B6F1FF3FF5D089
:10332800FEF7F6FBA0EB0800B04201D8002EEDD165
:1033380021684B6803F4804394F84220D2B288692C
:1033480010F4004F02D00BB9202A18D123689B69CA
:1033580013F0200FDAD1FEF7DBFBA0EB08001928E9
:10336800F4D9636C43F020036364202384F841306C
:10337800002384F8423084F840300125E6E74B68A2
:1033880043F480434B60FEF7C3FB8046DEE7002D25
:1033980040D12022DA610427012500E000252268B7
:1033A800936913F4807F05D047F001074FF48071CB
:1033B800D161012513F4806F06D047F00807226811
:1033C8004FF48061D161012513F4007F24D047F0C8
:1033D800020723684FF40072DA6101252046FFF7DF
:1033E80059FF2268536823F0FF7323F48B3323F4C7
:1033F800FF7323F001035360636C3B436364202332
:1034080084F84130002384F8423084F8403028465C
:10341800BDE8F0810427C2E7002DF8D0DEE770B5DB
:1034280004460D46164623689B6913F0020F1DD10A
:10343800324629462046FFF75CFFC8B9B5F1FF3F81
:10344800F1D0FEF765FB801BA84201D8002DEAD118
:10345800636C43F020036364202384F84130002325
:1034680084F8423084F84030012000E0002070BD2C
:103478000120FCE72DE9F0410646884617461D461F
:103488003468A46938EA04040CBF01240024BC424F
:1034980018D1B5F1FF3FF3D0FEF73AFB069BC01AEF
:1034A800A84201D8002DEBD1736C43F0200373645C
:1034B800202386F84130002386F8423086F84030D1
:1034C800012000E00020BDE8F08100002DE9F04176
:1034D80082B0044690461D46089E099F194B0093EA
:1034E8004FF08073EAB2FFF7E6FE3A4631462046CF
:1034F800FFF795FFF8B9012D0ED123685FFA88F21E
:103508009A6200973346002280212046FFF7B2FFD7
:10351800A8B902B0BDE8F08123684FEA18229A6280
:103528003A4631462046FFF77AFF30B923685FFAFA
:1035380088F29A62E5E70120EBE70120E9E701203C
:10354800E7E700BF002000802DE9F04182B0044683
:1035580090461D46089E099F184B00930023EAB227
:10356800FFF7A9FE3A4631462046FFF758FFF8B95B
:10357800012D0ED123685FFA88F29A6200973346CC
:10358800002240212046FFF775FFA8B902B0BDE828
:10359800F08123684FEA18229A623A46314620465B
:1035A800FFF73DFF30B923685FFA88F29A62E5E7D2
:1035B8000120EBE70120E9E70120E7E70020008090
:1035C80070B505460C4616462B689B6913F0200F0C
:1035D8001AD1324621462846FFF78BFEB0B9FEF7CE
:1035E80097FA801BA04201D8002CEDD16B6C43F0F8
:1035F80020036B64202385F84130002385F842308E
:1036080085F84030012070BD0020FCE70120FAE772
:10361800002859D010B5044690F84130002B43D00B
:10362800242384F841302268136823F001031360CF
:103638006368226823F0706313612268936823F437
:1036480000439360E368012B33D0A368226843F4F6
:1036580004439360E368022B31D02268536843F037
:10366800007343F4004353602268D36823F4004393
:10367800D360236962691343A169226843EA01237D
:10368800D360E369216A22680B43136022681368D8
:1036980043F00103136000206064202384F8413064
:1036A800206384F8420010BD80F84030FEF7F8F837
:1036B800B6E7A368226843F400439360CAE7236827
:1036C8004FF400625A60C8E7012070472DE9F04FB7
:1036D80083B00E46BDF834A00E9D90F84110C9B2D3
:1036E800202940F0BB800446904699460C9BCBB1FC
:1036F800BAF1000F16D090F84030012B00F0B280DC
:103708004FF0010B80F840B0FEF702FA0746009030
:1037180019235A464FF400412046FFF7ABFE30B15B
:1037280001209CE04FF400736364012097E021239B
:1037380084F84130402384F84230002363640C9AB3
:103748006262A4F82AA06363019700954B4642463B
:1037580031462046FFF7BAFE70B9638D9BB2FF2B46
:103768000FD9FF222285002300934FF08073314642
:103778002046FFF7A0FD21E0002384F8403058469A
:103788006DE0628D92B22285002300934FF00073A2
:10379800D2B231462046FFF78EFD0FE0628D92B21D
:1037A8002285002300934FF00073D2B231462046A1
:1037B800FFF781FD638D9BB2002B33D03A46294633
:1037C8002046FFF72CFE00284ED1626A2368127843
:1037D8009A62636A01336362638D9BB2013B9BB259
:1037E8006385238D013B9BB22385628D92B2002AAB
:1037F800E0D0002BDED100972B4600228021204606
:10380800FFF738FE90BB638D9BB2FF2BC6D9FF2212
:103818002285002300934FF0807331462046FFF73E
:103828004AFDC7E73A4629462046FFF7C9FEF8B9D8
:1038380023682022DA6121684B6823F0FF7323F4A0
:103848008B3323F4FF7323F001034B6084F841208A
:10385800002384F8423084F8403000E0022003B0AE
:10386800BDE8F08F0220FAE70120F8E70120F6E72B
:103878000120F4E72DE9F04F83B00E46BDF834A0DF
:103888000E9D90F84110C9B2202940F0BC80044632
:10389800904699460C9BCBB1BAF1000F16D090F820
:1038A8004030012B00F0B3804FF0010B80F840B09E
:1038B800FEF72EF90746009019235A464FF40041A7
:1038C8002046FFF7D7FD30B101209DE04FF400738B
:1038D8006364012098E0222384F84130402384F86F
:1038E8004230002363640C9A6262A4F82AA06363DE
:1038F800019700954B46424631462046FFF724FE85
:1039080070B9638D9BB2FF2B0FD9FF222285444BE0
:1039180000934FF0807331462046FFF7CCFC21E03E
:10392800002384F8403058466EE0628D92B22285BA
:103938003B4B00934FF00073D2B231462046FFF75D
:10394800BAFC0FE0628D92B22285002300934FF0FB
:103958000073D2B231462046FFF7ADFC638D9BB2AF
:10396800002B34D000972B46002204212046FFF775
:1039780081FD00284DD123685A6A636A1A70636A08
:1039880001336362228D013A92B22285638D9BB224
:10399800013B9BB26385638D9BB2002BDED0002A6E
:1039A800DCD100972B4680212046FFF763FD90BBB2
:1039B800638D9BB2FF2BC5D9FF222285002300937C
:1039C8004FF0807331462046FFF775FCC6E73A464C
:1039D80029462046FFF7F4FDF8B923682022DA616A
:1039E80021684B6823F0FF7323F48B3323F4FF73B0
:1039F80023F001034B6084F84120002384F842300F
:103A080084F8403000E0022003B0BDE8F08F0220C7
:103A1800FAE70120F8E70120F6E70120F4E700BF04
:103A2800002400802DE9F04385B01D460023039350
:103A380090F84130DBB2202B40F09E800646894644
:103A4800904603689B6913F4004F40F0978090F804
:103A58004030012B00F09480012380F8403024236B
:103A680080F841300023436444E0C9F3090343F07C
:103A7800007343F4005344E033689C69C4F3401472
:103A88009B69C3F30013C4B9BBB9B5F1FF3FF3D0C9
:103A9800FEF73EF8C01BA84201D8002DECD1202328
:103AA80086F84130736C43F020037364002386F872
:103AB8004030012005B0BDE8F08333689B6913F0FE
:103AC800100F2BD000972B46002220213046FFF7FD
:103AD800D1FC002858D133681022DA6133682022DB
:103AE800DA61039B43452AD0039B01330393039B6D
:103AF800434535D2F368012BB7D0C9F3090343F422
:103B0800205332685360FEF703F8074633689C6910
:103B1800C4F340149B69C3F30013B4E700972B4622
:103B2800002220213046FFF7A5FC58BB326820232D
:103B3800D36186F84130002386F84030BAE732680E
:103B4800536843F48043536000972B46002220219A
:103B58003046FFF78FFCC8B933682022DA61C3E723
:103B6800202386F84130736C43F0200373640023EC
:103B780086F8403001209DE702209BE7022099E764
:103B8800022097E7012095E7012093E7012091E7BC
:103B9800034690F84120D2B2202A23D190F8402041
:103BA800012A21D0012280F84020242280F84120D7
:103BB8000068026822F0010202601868026822F4B4
:103BC80080520260186802681143016019680A6827
:103BD80042F001020A60202283F84120002083F885
:103BE800400070470220704702207047034690F853
:103BF8004120D2B2202A21D190F84020012A1FD09A
:103C0800012280F84020242280F8412000680268C0
:103C180022F0010202601868026822F4706242EA27
:103C28000122026019680A6842F001020A60202233
:103C380083F84120002083F8400070470220704735
:103C48000220704730B4036A23F001030362026A5A
:103C58004468836923F4803323F073030D681D439C
:103C680022F002028B6813431C4A90420FD002F5DF
:103C7800006290420BD002F54062904207D002F5F4
:103C88008062904203D002F58062904205D123F011
:103C98000803CA681A4322F00403104A90420FD05E
:103CA80002F5006290420BD002F54062904207D0C4
:103CB80002F58062904203D002F58062904205D1FD
:103CC80024F440744A6922438C6914434460856132
:103CD8004A684263036230BC704700BF002C014051
:103CE80030B4036A23F480730362036A4468C269C8
:103CF80022F4803222F073020D68154323F4007316
:103D08008A6843EA0223184A904203D002F5006207
:103D1800904206D123F40063CA6843EA022323F4DD
:103D28008063114A90420FD002F5006290420BD096
:103D380002F54062904207D002F58062904203D0BB
:103D480002F58062904207D124F440524C6942EA5D
:103D580004128C6942EA04144460C5614A68C2636B
:103D6800036230BC704700BF002C014030B4036AC6
:103D780023F480530362036A4468C26922F08072A4
:103D880022F4E6420D6842EA052223F400538D68C6
:103D980043EA0533174DA84203D005F50065A8424C
:103DA80006D123F40043CD6843EA053323F4804366
:103DB800104DA8420FD005F50065A8420BD005F5B7
:103DC8004065A84207D005F58065A84203D005F5EF
:103DD8008065A84207D124F4404C4C694CEA841C05
:103DE8008C694CEA84144460C2614A6802640362C4
:103DF80030BC7047002C014030B4036A23F4803390
:103E08000362036A4468026D22F4803222F0700271
:103E18000D68154323F400338A6843EA02430F4AC6
:103E280090420FD002F5006290420BD002F540623A
:103E3800904207D002F58062904203D002F580627A
:103E4800904204D124F480344A6944EA022444604C
:103E580005654A688264036230BC7047002C0140E3
:103E680030B4036A23F480130362036A4468026D62
:103E780022F0807222F4E0420D6842EA052223F41F
:103E880000138D6843EA05530F4DA8420FD005F57E
:103E98000065A8420BD005F54065A84207D005F596
:103EA8008065A84203D005F58065A84204D124F4B2
:103EB80080244D6944EA8524446002654A68C264E6
:103EC800036230BC704700BF002C014010B4036A85
:103ED800046A24F001040462846924F0F00C4CEABA
:103EE800021223F00A030B43826103625DF8044B5C
:103EF800704710B4036A23F0100303628469036AED
:103F080024F4704C4CEA023223F0A00343EA011374
:103F1800826103625DF8044B7047836823F44013A1
:103F280023F070030B4343F00703836070470000DE
:103F380090F83D30DBB2012B32D1022380F83D30BE
:103F48000268D36843F00103D3600368174A9342B9
:103F580018D0B3F1804F15D0A2F59432934211D006
:103F680002F5806293420DD002F59632934209D051
:103F780002F54062934205D01A6842F001021A60C5
:103F88000020704799680A4A0A40062A0AD0B2F502
:103F9800803F09D01A6842F001021A600020704779
:103FA800012070470020704700207047002C014016
:103FB80007000100704770477047704770477047A7
:103FC80010B5044603681A6912F0020F12D0DA68B5
:103FD80012F0020F0ED06FF002021A61012303776C
:103FE80003689B6913F0030F00F09F80FFF7E5FF5C
:103FF8000023237723681A6912F0040F13D0DA68B4
:1040080012F0040F0FD06FF004021A610223237715
:1040180023689B6913F4407F00F08D802046FFF7EA
:10402800CCFF0023237723681A6912F0080F12D0F7
:10403800DA6812F0080F0ED06FF008021A61042334
:1040480023772368DB6913F0030F7BD02046FFF743
:10405800B4FF0023237723681A6912F0100F12D0D7
:10406800DA6812F0100F0ED06FF010021A610823F0
:1040780023772368DB6913F4407F6AD02046FFF773
:104088009CFF0023237723681A6912F0010F03D0DD
:10409800DA6812F0010F63D123681A6912F0800FF1
:1040A80003D0DA6812F0800F61D123681A6912F41C
:1040B800807F03D0DA6812F0800F5FD123681A6915
:1040C80012F0400F03D0DA6812F0400F5DD1236878
:1040D8001A6912F0200F03D0DA6812F0200F5BD1B2
:1040E80023681A6912F4801F03D0DA6812F4801F5B
:1040F80059D123681A6912F4001F03D0DA6812F440
:10410800001F57D123681A6912F4800F03D0DA68A8
:1041180012F4800F55D123681A6912F4000F03D0E6
:10412800DA6812F4000F53D110BDFFF745FF20469F
:10413800FFF744FF5CE72046FFF73EFF2046FFF706
:104148003DFF6EE72046FFF737FF2046FFF736FFB3
:104158007FE72046FFF730FF2046FFF72FFF90E765
:104168006FF001021A612046FFF725FF94E76FF010
:1041780080021A61204600F086FB96E76FF4807291
:104188001A61204600F080FB98E76FF040021A6140
:104198002046FFF714FF9AE76FF020021A612046C5
:1041A80000F070FB9CE76FF480121A61204600F063
:1041B8006CFB9EE76FF400121A61204600F066FB64
:1041C800A0E76FF480021A61204600F060FBA2E7C6
:1041D8006FF400021A61204600F05AFBA4E70000C1
:1041E80003682C4A90420ED0B0F1804F0BD0A2F554
:1041F8009432904207D002F58062904203D002F5D3
:104208009632904203D123F070034A681343214A3F
:1042180090421AD0B0F1804F17D0A2F59432904254
:1042280013D002F5806290420FD002F59632904288
:104238000BD002F54062904207D002F580629042AE
:1042480003D002F58062904203D123F44073CA6818
:10425800134323F080034A69134303608B68C362E6
:104268000B6883620B4B98420FD003F500639842AA
:104278000BD003F54063984207D003F5806398425A
:1042880003D003F58063984201D10B6903630123CE
:1042980043617047002C014060B310B5044690F8A4
:1042A8003D3013B3022384F83D30214651F8040B06
:1042B800FFF796FF012384F8483084F83E3084F8ED
:1042C8003F3084F8403084F8413084F8423084F834
:1042D800433084F8443084F8453084F8463084F814
:1042E800473084F83D30002010BD80F83C30FDF7A1
:1042F80031FBD7E70120704760B310B5044690F84A
:104308003D3013B3022384F83D30214651F8040BA5
:10431800FFF766FF012384F8483084F83E3084F8BC
:104328003F3084F8403084F8413084F8423084F8D3
:10433800433084F8443084F8453084F8463084F8B3
:10434800473084F83D30002010BD80F83C30FFF73E
:1043580031FED7E70120704730B4036A23F0100319
:104368000362036A4468826922F0807222F4E6429A
:104378000D6842EA052223F020038D6843EA0513FD
:10438800174DA84203D005F50065A84206D123F0D1
:104398008003CD6843EA051323F04003104DA8427B
:1043A8000FD005F50065A8420BD005F54065A84279
:1043B80007D005F58065A84203D005F58065A842B9
:1043C80007D124F4406C4C694CEA840C8C694CEAA3
:1043D8008404446082614A688263036230BC704727
:1043E800002C014038B590F83C30012B00F0958046
:1043F80004460D46012380F83C30142A00F28880D8
:10440800DFE802F00B8686861F86868634868686D7
:10441800488686865D86868671000068FFF712FCEE
:104428002268936943F0080393612268936923F033
:10443800040393612268936929690B4393610020FF
:1044480067E00068FFF788FF2268936943F4006318
:1044580093612268936923F4806393612268936966
:10446800296943EA01239361002052E00068FFF7BD
:1044780037FC2268D36943F00803D3612268D36903
:1044880023F00403D3612268D36929690B43D361FC
:1044980000203EE00068FFF769FC2268D36943F416
:1044A8000063D3612268D36923F48063D3612268EF
:1044B800D369296943EA0123D361002029E0006810
:1044C800FFF79AFC2268136D43F00803136522680E
:1044D800136D23F0040313652268136D29690B43D8
:1044E8001365002015E00068FFF7BAFC2268136D19
:1044F80043F4006313652268136D23F48063136526
:104508002268136D296943EA01231365002000E03E
:104518000120002384F83C3038BD0220FCE710B4A9
:10452800846824F47F4C42EA03220A4342EA0C02DC
:1045380082605DF8044B704790F83C30012B00F026
:104548008F8010B50446012380F83C30022380F8A0
:104558003D3002689068434B034093600B68702BB2
:1045680055D031D8502B6CD00CD9602B2AD1CA68C1
:1045780049682068FFF7BDFC60212068FFF7CDFC83
:10458800002035E0402B0AD1CA6849682068FFF747
:104598009DFC40212068FFF7C0FC002028E05BD884
:1045A800202B07D003D9302B04D0012020E00BB1F9
:1045B800102B05D119462068FFF7AFFC002017E043
:1045C800012015E0012013E0B3F5005F2CD00BD9D2
:1045D800254A9342EED012D9244A9342EAD0303287
:1045E8009342E7D0012003E0B3F5805F36D1002085
:1045F800012384F83D30002384F83C3010BDB3F12A
:10460800101FD7D0103A9342D4D00120F0E7CB68DE
:104618004A6889682068FFF782FF2268936843F038
:10462800770393600020E3E7CB684A6889682068CD
:10463800FFF775FF2268936843F480439360002076
:10464800D6E7CA6849682068FFF740FC502120680F
:10465800FFF763FC0020CBE70120C9E70120C7E78B
:10466800022070478800CEFF300010004000100084
:1046780001F01F014FF0010C0CFA01FC036A23EA58
:104688000C030362036A8A40134303627047000005
:1046980010B5044610293CD8DFE801F0093B3B3B44
:1046A8001F3B3B3B263B3B3B2D3B3B3B340090F8C1
:1046B8003E30DBB2013B18BF0123002B40F08E8057
:1046C800102979D8DFE801F02C787878687878783C
:1046D8006C78787870787878740090F83F30DBB22E
:1046E800013B18BF0123E8E790F84030DBB2013BFB
:1046F80018BF0123E1E790F84130DBB2013B18BF56
:104708000123DAE790F84230DBB2013B18BF0123FE
:10471800D3E790F84330DBB2013B18BF0123CCE765
:10472800022384F83E3001222068FFF7A1FF2368A6
:104738002D4A93420FD002F5006293420BD002F546
:104748004062934207D002F58062934203D002F59B
:104758008062934203D15A6C42F400425A6423683F
:10476800214A93422CD0B3F1804F29D0A2F594323C
:10477800934225D002F58062934221D002F5963209
:1047880093421DD002F54062934219D01A6842F054
:1047980001021A60002022E0022384F83F30C2E7B9
:1047A800022384F84030BEE7022384F84130BAE798
:1047B800022384F84230B6E7022384F84330B2E794
:1047C80099680A4A0A40062A0AD0B2F5803F09D0F9
:1047D8001A6842F001021A60002000E0012010BDB2
:1047E8000020FCE70020FAE7002C01400700010048
:1047F80090F83C20012A40D030B40346012280F8CA
:104808003C20022280F83D200068426884681C4DE4
:10481800A84203D005F50065A84203D122F470022E
:104828004D682A4322F0007222F070020D682A4374
:1048380042601A681248824212D0B2F1804F0FD0FB
:10484800A0F5943082420BD000F58060824207D0F8
:1048580000F59630824203D000F54060824204D1D0
:1048680024F08004896821439160012283F83D2067
:10487800002083F83C0030BC70470220704700BF1E
:10488800002C014070477047704770477047704769
:104898007047000070B504460168836802691343D5
:1048A80042691343C269134308688B4A02401A439A
:1048B8000A602268536823F44053E1680B4353604D
:1048C800A1692268854B9A4201D0236A19439368EB
:1048D80023F06E4323F430630B4393602268D36A5A
:1048E80023F00F03616A0B43D36223687C4A934227
:1048F80023D07C4A934234D07B4A93424AD07B4AA5
:10490800934259D0754A934268D0102273498B421A
:1049180000F09580E069B0F5004F00F0D280082AD9
:1049280000F24F81DFE812F01201340110014D014D
:1049380037014D014D014D013A0102F55842D2F8B7
:10494800882002F00302032A09D8DFE802F00204F3
:104958005C060122DAE70422D8E70822D6E710220B
:10496800D4E702F5E632D2F8882002F00C020C2ACD
:104978000ED8DFE802F0070D0D0D090D0D0D4A0DDB
:104988000D0D0B000022C1E70422BFE70822BDE796
:104998001022BBE702F5E432D2F8882002F0300298
:1049A800202A34D004D8A2B3102A34D10422ADE787
:1049B800302A32D10822A9E702F5E232D2F888205B
:1049C80002F0C002802A2AD004D852B3402A2AD141
:1049D80004229BE7C02A28D1082297E702F5C832AB
:1049E800D2F8882002F44062B2F5006F1FD005D8D3
:1049F800FAB1B2F5806F1ED1042287E7B2F5406F95
:104A08001BD1082282E7022280E702227EE70222E7
:104A18007CE700227AE7102278E7102276E7022264
:104A280074E7002272E7102270E710226EE7022274
:104A38006CE700226AE7102268E7102266E7082A76
:104A480000F2AF80DFE802F008AD3BAD38ADADADA8
:104A580005004FF4004004E0FDF788FC002800F052
:104A6800A280626A224B33F81220B0FBF2F3656829
:104A780005EB4501994200F29880B3EB053F00F23F
:104A88009680002633463146FCF772F8090241EA5F
:104A9800106100026B08C0182A46334641F1000134
:104AA800FCF766F8A0F54072124B9A4200F281803A
:104AB8002368D860304662E0FDF712FBCEE70E4867
:104AC800CFE7082A77D8DFE802F0193905763C766F
:104AD80076761D00084815E0F369FFCF0080004096
:104AE800003801400044004000480040004C0040AD
:104AF80008800008FFFC0F000024F400FDF736FCD6
:104B080000285AD0626A324B33F81230B0FBF3F007
:104B18006268530803EB4003B3FBF2F3A3F11001FF
:104B28004FF6EF7291424AD89AB222F00F02C3F3BD
:104B3800420313432268D360002020E0FDF728FCDD
:104B4800DEE7FDF7CDFADBE7224803E0FDF70EFCD0
:104B5800002838D0626A1E4B33F81230B0FBF3F0ED
:104B6800636800EB5300B0FBF3F0A0F110024FF6BE
:104B7800EF739A4229D8236880B2D86000200123B5
:104B8800A4F86A30A4F8683000232367636770BD0F
:104B9800FDF7FEFBDCE7FDF7A3FAD9E74FF4004089
:104BA800D8E70120EBE70020E9E70120E7E701204B
:104BB800E5E70120E3E70120E1E70020DFE7012046
:104BC800DDE70120DBE70020D9E70120D7E700BFB8
:104BD800088000080024F400836A13F0010F06D04F
:104BE8000268536823F40033C16A0B435360836A35
:104BF80013F0020F06D00268536823F48033016B68
:104C08000B435360836A13F0040F06D0026853689D
:104C180023F48023416B0B435360836A13F0080F1E
:104C280006D00268536823F40043816B0B4353603A
:104C3800836A13F0100F06D00268936823F4805338
:104C4800C16B0B439360836A13F0200F06D0026890
:104C5800936823F40053016C0B439360836A13F049
:104C6800400F0AD00268536823F48013416C0B4349
:104C78005360436CB3F5801F0BD0836A13F0800F29
:104C880006D00268536823F40023C16C0B435360B9
:104C980070470268536823F4C003816C0B43536068
:104CA800EBE72DE9F84305460F4616469946DDF829
:104CB80020802B68DC6937EA04040CBF0124002437
:104CC800B44257D1B8F1FF3FF3D0FCF721FFA0EB76
:104CD800090040452FD8B8F1000F2CD02B681A686E
:104CE80012F0040FE5D0DA6912F4006FE1D04FF446
:104CF80000621A622A6852E8003F23F4D07342E83F
:104D080000310029F6D12A6802F1080353E8003F70
:104D180023F00103083242E800310029F3D12023AF
:104D2800C5F88430C5F88830C5F88C30002385F87C
:104D3800803003201FE02A6852E8003F23F4D07334
:104D480042E800310029F6D12A6802F1080353E845
:104D5800003F23F00103083242E800310029F3D173
:104D68002023C5F88430C5F88830002385F88030C2
:104D7800032000E00020BDE8F88330B583B0044686
:104D88000023C0F88C30FCF7C3FE05462268126881
:104D980012F0080F0FD123681B6813F0040F18D105
:104DA8002023C4F88430C4F888300020E06684F8F2
:104DB800800003B030BD6FF07E43009303460022AD
:104DC8004FF400112046FFF76CFF0028E3D00320C2
:104DD800EFE76FF07E4300932B4600224FF48001EB
:104DE8002046FFF75EFF0028DAD00320E1E778B31A
:104DF80010B50446D0F884300BB32423C4F88430AB
:104E08002268136823F0010313602046FFF742FD70
:104E1800012813D0A36ABBB92268536823F49043CE
:104E280053602268936823F02A039360226813680A
:104E380043F0010313602046FFF79FFF10BD80F881
:104E48008030FCF7DDFDD8E72046FFF7C5FEE3E735
:104E580001207047436E2BB90123A0F86A30A0F8EF
:104E68006830704730B403689A68C2F34262996840
:104E7800490F094D6B5CDB00084C615C93FBF1F357
:104E8800A0F86A30AB5CDB00A25C93FBF2F3A0F8FD
:104E9800683030BC704700BF2880000820800008B8
:104EA80090F88030012B18D0012380F8803024231B
:104EB800C0F8843003681A68196821F00101196084
:104EC80022F000520023436601680A602022C0F8DD
:104ED800842080F88030184670470220704738B523
:104EE80090F88030012B1DD00446012380F88030D3
:104EF8002423C0F8843003681D681A6822F0010270
:104F08001A600268936823F0604319439160FFF7C1
:104F1800A1FF23681D602023C4F88430002084F892
:104F2800800038BD0220FCE738B590F88030012BAE
:104F38001DD00446012380F880302423C0F8843033
:104F480003681D681A6822F001021A6002689368F3
:104F580023F0606319439160FFF77CFF23681D60AD
:104F68002023C4F88430002084F8800038BD022053
:104F7800FCE70000034AD2F8883043F47003C2F813
:104F88008830704700ED00E008B500220F4910484E
:104F980002F061F970B90F490D4802F073F960B970
:104FA8000D490B4802F0EFFF50B9094802F081F9AA
:104FB80048B908BDFBF792FFEDE7FBF78FFFEFE776
:104FC800FBF78CFFF1E7FBF789FFF2E740000020D1
:104FD800A4030020F800002060000020032805D862
:104FE800DFE800F005040205012070470320704740
:104FF80008B5FCF727F908BD10B592B0044644225D
:10500800002101A8FBF74CF92268114B9A4201D004
:1050180012B010BD4FF40053019301A8FDF7CAF96F
:1050280090B90C4B9A6D42F400029A659B6D03F49B
:1050380000030093009B002211461420FDF7F8FCA2
:105048001420FDF705FDE3E7FBF748FFE9E700BF9C
:10505800005C00400010024008B500F52C71D0F843
:10506800F00202F03BF908BD08B501EB810300EB43
:10507800C303D3F87C21D0F8F00202F05BF908BD35
:1050880008B501EB810300EBC303DA6BD0F8F0023B
:1050980002F08CF908BD08B5D0F8F00202F02CFA3D
:1050A80008BD10B504468368022B09D10121D4F844
:1050B800F00202F007FAD4F8F00202F0D6F910BDB7
:1050C800FBF70CFFF2E7000010B50446D0F8F00239
:1050D80002F0FBF9A36923B1024A136943F00603FE
:1050E800136110BD00ED00E010B50446836923B9D3
:1050F800D4F8F00202F0F3F910BD044A136923F062
:1051080006031361FFF774FFF2E700BF00ED00E04C
:1051180010B504461648C0F8F042C4F8C402154B4E
:105128000360082343600223836003610023436113
:105138008361C361036200F0DFF9B0B91023002274
:105148001146D4F8C40201F015F950230022802139
:10515800D4F8C40201F00EF9074B01221146D4F825
:10516800C40201F007F9002010BDFBF7B7FEE5E720
:1051780048220020005C00409000500108B5D0F89B
:10518800C40200F02BFAFFF729FF08BD08B59446C2
:105198001A466346D0F8C40200F0B5FFFFF71EFFB9
:1051A80008BD08B5D0F8C40200F0EFFFFFF716FFFE
:1051B80008BD08B5D0F8C40201F06CF8FFF70EFF7F
:1051C80008BD08B5D0F8C40201F099F8FFF706FF4A
:1051D80008BDD0F8C43211F0800F08D101F07F016A
:1051E80001EB810103EBC10393F86A01704701F0F9
:1051F8007F01013101EB810103EBC103987870470E
:1052080008B5D0F8C40200F091FEFFF7E7FE08BD2C
:1052180008B5D0F8C40201F015F8FFF7DFFE08BDA5
:1052280008B5D0F8C40200F0E2FFFFF7D7FE08BDCA
:1052380008B5D0F8C40200F0FCFF08BD10B504465C
:1052480011B101290FD010BD836923B9D4F8F00238
:1052580002F045F9F7E7FFF7CBFE094A136923F097
:1052680006031361F2E7D0F8F00202F02EF9A36901
:10527800002BE8D0024A136943F006031361E2E702
:1052880000ED00E0004870477406002070470000F9
:1052980012230B80004870472C00002004230B8049
:1052A8000048704728000020002393421ED200B512
:1052B80010E00CF1370C01F813C000014FEA430C61
:1052C8000CF1010C4FF0000E01F80CE00133DBB2D9
:1052D800934209D24FEA107CB0F1204FE9D20CF189
:1052E800300C01F813C0E8E75DF804FB70470000D4
:1052F80038B50B4BD3F89005D3F89445D3F89835C7
:10530800C01800D138BD074D08222946FFF7CCFF49
:10531800042205F110012046FFF7C6FFF2E700BF9F
:105328000070FF1F0E00002008B51A230B80FFF73E
:10533800DFFF014808BD00BF0C00002008B50A4681
:1053480028B90549054802F030FC034808BD024960
:10535800024802F02AFCF8E73C25002048800008B3
:1053680010B50A46034C2146034802F01EFC2046AD
:1053780010BD00BF3C2500205C80000808B50A4627
:1053880028B90549054802F010FC034808BD024940
:10539800024802F00AFCF8E73C250020708000086B
:1053A80008B50A4628B90549054802F0FEFB034836
:1053B80008BD0249024802F0F8FBF8E73C25002046
:1053C8008080000800207047002070470020704748
:1053D8000020704700207047002070470020704769
:1053E80038B512F4804F43D00468B4F8503091F8BF
:1053F80000C04FEACC0E1EFA83F32344B3F80244EC
:10540800C4F309048B69A34228D31B1B8B618B69E6
:105418007BB9056835F82C309BB223F4804323F020
:10542800700383F4005343F4004343F0800325F8EA
:105438002C3012F0400F0ED002680D7832F825306B
:105448009BB223F4E04323F0700343F4004343F09A
:10545800C00322F8253024B9204638BD00238B61CB
:10546800D5E723460A894969006801F0DCFEF3E7BD
:105478000468B4F8503091F800C04FEACC0E1EFA18
:1054880083F32344B3F80644C4F309048B69A342A5
:105498002FD31B1B8B618B697BB9056835F82C30C2
:1054A8009BB223F4804323F0700383F4005343F446
:1054B800004343F0800325F82C3012F0400F0FD141
:1054C800026891F800C032F82C309BB223F4E04314
:1054D80023F0700343F4004343F0C00322F82C3058
:1054E800002CB9D023464A894969006801F09BFE1F
:1054F800B2E700238B61CEE700286DD030B587B0C6
:10550800044690F8A9323BB1032384F8A9322068F5
:1055180000F06BFF00231FE080F8A832FFF76CFD56
:10552800F2E75A1C02EB820104EBC101012048702A
:1055380002EB820104F8313003EB830104EBC10173
:10554800CB8602EB820C04EBCC0C00208CF8030019
:105558008863C8630864D3B260688342E1D30023D8
:1055680016E003EB830204EBC202002182F8691102
:1055780082F8683182F86B11C2F87811C2F87C1190
:1055880003EB830204EBC202C2F880110133DBB2E1
:105598009842E6D8A4465CF8105BEE46BCE80F00DB
:1055A800AEE80F00DCF80030CEF80030231D0ECB3B
:1055B800284600F024FF002384F82430012384F8CF
:1055C800A932E369012B02D0002007B030BD204684
:1055D80000F0ECFE0020F8E70120704790F8A832B0
:1055E800012B0ED010B50446012380F8A8320068BC
:1055F80000F0F2FE206801F045FA002084F8A802C5
:1056080010BD0220704770B505460C46164612F0CC
:10561800400F00F009810268B2F850300978C800DC
:1056280010FA83F31344B3F80224C2F30902A369FE
:10563800934251D99B1AA361A369002B68D163785F
:10564800002B4CD12A68B2F8503012FA83F3034485
:10565800B3F8022492B222F4F84292B2A3F80224D8
:10566800B3F802246FEA42426FEA524292B2A3F8B8
:1056780002242A686378002B3DD1B2F8503012FA20
:1056880083F3227803EBC203B3F8062492B222F420
:10569800F84292B2A3F80624B3F806246FEA42420D
:1056A8006FEA524292B2A3F8062421782846FFF7FF
:1056B800E7FC16F4804F40D02A68217832F8213070
:1056C8009BB223F4E04323F0700343F4404343F0D8
:1056D800800322F8213030E00023A361ACE7012BDE
:1056E800C7D12A68B2F8503012FA83F30344002273
:1056F800A3F80224BDE7012BD7D1B2F8503012FA33
:1057080083F3227803EBC2030022A3F80624CCE734
:1057180016F4804F0DD0286830F821309BB223F45E
:10572800E04323F0700343F4404343F0800320F840
:10573800213094F82430012B12D02A68217832F8CD
:1057480021309BB223F4E04323F0400383F030037D
:1057580043F4004343F0800322F82130002070BD59
:10576800636913446361E3691344E361216A23694C
:1057780099421BD3C91A21626278002A3FD129684D
:10578800B1F8502011FA82F2217802EBC1023E2BC7
:1057980018D9590913F01F0F00D101396FEAC161F7
:1057A8006FEA514189B2A2F802142AE021B9002314
:1057B80084F824301346DFE7002384F8243023627A
:1057C8000B46D9E78BB9B2F8021489B221F4F84133
:1057D80089B2A2F80214B2F802146FEA41416FEAE2
:1057E800514189B2A2F802140BE0590813F0010FD5
:1057F80000D00131890289B2A2F8021401E0012A1D
:1058080006D09BB222896169286801F04AF994E7B9
:105818002968B1F8502011FA82F2217802EBC1020E
:1058280099B2A2F80214ECE70268B2F8503009788D
:10583800C80010FA83F31344B3F80624C2F309022C
:10584800A369934252D39B1AA361A369002B69D120
:105858006378002B4DD12A68B2F8503012FA83F3DE
:105868000344B3F8022492B222F4F84292B2A3F8A5
:105878000224B3F802246FEA42426FEA524292B21B
:10588800A3F802242A686378002B3ED1B2F850307E
:1058980012FA83F3227803EBC203B3F8062492B218
:1058A80022F4F84292B2A3F80624B3F806246FEA69
:1058B80042426FEA524292B2A3F80624217828465F
:1058C800FFF7DEFB16F4804F7FF437AF2A682178A4
:1058D80032F821309BB223F4E04323F0700343F401
:1058E800404343F0800322F8213026E70023A361D8
:1058F800ABE7012BC6D12A68B2F8503012FA83F30D
:1059080003440022A3F80224BCE7012BD6D1B2F845
:10591800503012FA83F3227803EBC2030022A3F873
:105928000624CBE716F4804F0DD1286830F82130D3
:105938009BB223F4E04323F0700343F4404343F065
:10594800800320F8213094F82430012B7FF4F5AE41
:10595800636913446361E3691344E361216A23695A
:1059680099421BD3C91A216229686278002A3ED15C
:10597800B1F8502011FA82F2217802EBC1023E2BD5
:1059880018D9590913F01F0F00D101396FEAC16105
:105998006FEA514189B2A2F806142AE021B900231E
:1059A80084F824301346DFE70023236284F8243088
:1059B8000B46D9E78BB9B2F8061489B221F4F8413D
:1059C80089B2A2F80614B2F806146FEA41416FEAE8
:1059D800514189B2A2F806140BE0590813F0010FDF
:1059E80000D00131890289B2A2F8061401E0012A27
:1059F80006D09BB262896169286801F052F89CE67A
:105A0800B1F8502011FA82F2217802EBC10299B262
:105A1800A2F80614EDE72DE9F0410546CAE003882F
:105A28009BB223F4E14323F070036FEA43436FEA28
:105A380053439BB203802968B1F8503095F8282069
:105A4800D20012FA83F30B44B3F80234C3F3090308
:105A58006B64EA6B1A44EA6300212846FFF710FBDF
:105A680095F82430002B00F0A5802B6C002B40F01B
:105A7800A18095F824302A6843F08003A2F84C30BE
:105A8800002385F8243095E0B0F8503095F8682167
:105A9800D20012FA83F30344B3F80634C3F30903BC
:105AA800C5F88431B5F86E2105F52C7101F0BBFB02
:105AB8002A68138823F070031B051B0D43F080032D
:105AC80013802846FFF7C8FA74E089B9B3F80624AA
:105AD80092B222F4F84292B2A3F80624B3F806244C
:105AE8006FEA42426FEA524292B2A3F80624BFE03C
:105AF8004A0811F0010F00D00132920292B2A3F8C5
:105B08000624B5E030F824309EB213F4004F40F07C
:105B1800BE8016F0800F4DD0621C02EB820105EBAF
:105B2800C101286830F824309BB223F4E14323F004
:105B380070036FEA43436FEA53439BB220F8243063
:105B4800CB78022B00F0A78104EB840305EBC30399
:105B580000221A6493F8343023B316F0400F00F093
:105B680063814B78002B40F04C812A68B2F85030A2
:105B780012FA83F3621C02EB820215F8322003EB5F
:105B8800C203B3F8022492B222F4F84292B2A3F804
:105B98000224B3F802246FEA42426FEA524292B2F8
:105BA800A3F80224013404EB840415F834102846C1
:105BB800FFF766FA2868B0F8443013F4004F00F095
:105BC800B281B0F84440A3B214F00F049AD113F094
:105BD800100F3FF424AF03889AB213F4006F7FF4D8
:105BE80053AF12F4004FE5D0038823F070031B0570
:105BF8001B0D43F0800303802868B0F8503095F8F7
:105C08006821D20012FA83F30344B3F80634C3F3CD
:105C18000903C5F884318BB1D5F87C1171B1B5F899
:105C28006E2101F000FBD5F87C31D5F884211344AE
:105C3800C5F87C3100212846FFF716FA2B681A8828
:105C480012F4006FB6D1B3F8502013FA82F3D5F8E6
:105C580078113E297FF639AF4A0911F01F0F00D19C
:105C6800013A6FEAC2626FEA524292B2A3F806247E
:105C78002A6813889BB223F4804323F0700383F4CB
:105C8800405343F4004343F08003138092E730F815
:105C9800243023F070031B051B0D43F0800320F80C
:105CA800243004EB8401C90001F5B47105EB010847
:105CB80004EB840305EBC30393F87431002B40D144
:105CC8002868B0F8503004EB840205EBC20292F861
:105CD8006821D20012FA83F30344B3F80674C7F3B9
:105CE800090717BB04EB840305EBC303D3F884212E
:105CF8003A44C3F88421D3F87C213A44C3F87C2180
:105D0800D3F880313BB104EB840305EBC303D3F82C
:105D180078319F4270D204EB840305EBC30393F8F8
:105D280068112846FFF7A0F9F3E604EB840105EBB8
:105D3800C1013B46B1F86E21D1F87C1101F073FA2C
:105D4800D0E704EB840305EBC30393F86B31022B14
:105D580033D0296804EB840205EBC20292F868018B
:105D680031F820309BB223F4E04323F0700343F46E
:105D7800004343F0C00321F82030286892F86831C6
:105D880030F8232012F4804F1ED0B0F85020DB00EA
:105D980013FA82F30344B3F80274C7F30907002F18
:105DA800A0D004EB840105EBC1013B46B1F870219A
:105DB800D1F87C1101F037FA94E73246414628467B
:105DC800FFF70EFB07468DE7B0F85020DB0013FA0B
:105DD80082F30344B3F80674C7F30907002F81D090
:105DE80004EB840105EBC1013B46B1F87221D1F8FF
:105DF8007C1101F018FA75E74146286800F063FE47
:105E080087E6012B7FF4CEAE2A68B2F8503012FA3A
:105E180083F3621C02EB820215F8322003EBC20303
:105E28000022A3F80224BDE62A68631C03EB83035F
:105E380005EBC3035B78E3B9B2F8503012FA83F389
:105E4800621C02EB820215F8322003EBC203B3F89E
:105E5800062492B222F4F84292B2A3F80624B3F8C8
:105E680006246FEA42426FEA524292B2A3F806242D
:105E780098E6012B7FF496AEB2F8503012FA83F30D
:105E8800621C02EB820215F8322003EBC2030022E7
:105E9800A3F8062486E616F4807F3FD12868B0F878
:105EA8005030621C02EB820215F83260F20012FADE
:105EB80083F30344B3F80234C3F3090304EB840205
:105EC80005EBC202126C9A4210D904EB840705EB69
:105ED800C707D21A3A6404EB840205EBC202126CBB
:105EE8005AB931462846FFF7CBF863E604EB84023B
:105EF80005EBC20200271764EDE704EB840205EB0B
:105F0800C202D66B1E44D663526C04EB840405EBC4
:105F1800C4041344636400F0D6FD4BE632462846B9
:105F2800FFF771FB46E60020BDE8F08190F8A83243
:105F3800012B0DD010B50446012380F8A83280F853
:105F48002410006800F098FD002084F8A80210BD15
:105F58000220704710B50446006800F09EFD10F45A
:105F6800004F23D110F4806F24D110F4804F32D128
:105F780010F4005F39D110F4805F40D110F4006F45
:105F880067D110F0800F40F0818010F4007F40F05E
:105F9800AD8010F4807F27D02268B2F844309BB2DD
:105FA80023F480739BB2A2F844301DE02046FFF72B
:105FB80032FD19E02268B2F844309BB223F48063C2
:105FC8009BB2A2F844302046FFF76BF80021204628
:105FD800FFF7ACFF08E02268B2F844309BB223F424
:105FE80080439BB2A2F8443010BD2268B2F8443016
:105FF8009BB223F400539BB2A2F84430F4E7226822
:10600800B2F840309BB223F004039BB2A2F84030B0
:106018002268B2F840309BB223F008039BB2A2F882
:10602800403094F8E032012B0CD02046FFF75CF8A2
:106038002268B2F844309BB223F480539BB2A2F892
:106048004430D1E7002184F8E0122046FFF7F6F843
:10605800EBE72268B2F840309BB243F00803A2F89D
:1060680040302268B2F844309BB223F400639BB2FC
:10607800A2F844302268B2F840309BB243F00403DF
:10608800A2F840302046FFF71FF8ADE72268B2F8C3
:1060980044309BB223F080039BB2A2F8443094F8BA
:1060A800E032FBB92268B2F840309BB243F00403F7
:1060B800A2F840302268B2F840309BB243F008039F
:1060C800A2F84030012184F8E0122368B3F8543074
:1060D800C3F38D0303F03C03C4F8E4322046FFF712
:1060E800ADF881E72046FEF7EFFF7DE72268B2F8BA
:1060F80044309BB223F400739BB2A2F8443020468C
:10610800FEF7C9FF70E710B504468C4611F0800F02
:106118002AD101F0070000EB8001C90001F5B47E27
:1061280004EB0E0100EB800004EBC0004FF0000E02
:1061380080F869E10CF0070C81F800C00A61CB70A7
:106148004A780AB1A1F80EC0022B19D094F8A832E7
:10615800012B18D0012384F8A832206800F060F9D8
:10616800002084F8A80210BD01F00700013000EB00
:10617800800104EBC1014FF0010E81F801E0D9E77D
:1061880000230B71E2E70220EDE710B504460B4649
:1061980011F0800F1FD101F0070202EB8201C90044
:1061A80001F5B471014402EB820200EBC202002047
:1061B80082F8690103F007030B7094F8A832012BE9
:1061C80013D0012384F8A832206800F0F4FA0020E4
:1061D80084F8A80210BD01F00702013202EB820127
:1061E80000EBC10101204870E4E70220F2E710B596
:1061F80001F0070404EB8401C90001F5B4710144FE
:1062080004EB840C00EBCC0CCCF87C21CCF880316E
:106218000023CCF884318CF869318CF8684124B9B2
:10622800006800F050FC002010BD006800F04BFC36
:10623800F9E701F0070101EB810100EBC100D0F89B
:106248008401704710B501F0070404F1010C0CEB50
:106258008C0100EBC10104EB840E00EBCE0ECEF8EE
:106268003C20CEF8403001228EF84C20CEF8483041
:106278000023CEF844304A700CEB8C0C00F83C40FC
:1062880024B9006800F01FFC002010BD006800F071
:106298001AFCF9E70B4601F0070241688A422AD83E
:1062A80010B5044613F0800F1DD103EB8301C9001C
:1062B80001F5B471014403EB830300EBC303002031
:1062C80083F8690101238B700A7094F8A832012BB6
:1062D80013D0012384F8A832206800F057FB00206F
:1062E80084F8A80210BD531C03EB830100EBC10125
:1062F80001204870E6E7012070470220F2E70B46CC
:1063080001F00F014268914230D810B5044613F0ED
:10631800800F21D103F0070202EB8201C90001F5C9
:10632800B471014402EB820200EBC202002082F841
:10633800690100228A7003F007030B7094F8A832F1
:10634800012B15D0012384F8A832206800F043FB04
:10635800002084F8A80210BD03F00702013202EB06
:10636800820100EBC10101204870E2E7012070477B
:106378000220F0E711F0800F0BD001F00701013186
:1063880001EB810100EBC10052B90273C380002008
:10639800704701EB8101C90001F5B4710844F3E7C6
:1063A8000122027303811B0C4381F0E70346026854
:1063B8000121C0F8E812002083F8E002B2F8543056
:1063C8009BB20B43A2F85430B2F854309BB243F05E
:1063D8000203A2F85430704703460020A3F8440093
:1063E8004BF68072A3F840207047B0F8403023F491
:1063F8007E535B045B0CA0F840300020704784B0EB
:10640800844601A880E80E000123ACF84030002043
:10641800ACF84000ACF84400ACF8500004B0704749
:1064280010B5034691F800C030F82C2092B222F43F
:10643800EC4222F0700292B2C878032861D8DFE8F3
:1064480000F0555C0258002048F2800E42EA0E0225
:1064580023F82C2091F800C033F82C2092B222F4B3
:10646800E04222F070024CEA020242EA0E0223F8ED
:106478002C200A7B002A40F0C2804A78002A51D09A
:10648800B3F8502013FA82F20C7802EBC402B1F888
:1064980006C04FEA5C0C4FEA4C0CA2F800C40C781A
:1064A80033F8242012F0400F0CD033F8242092B295
:1064B80022F4E04222F0700242F4004242F0C002AC
:1064C80023F82420CA78012A1DD0097833F821201E
:1064D80092B222F4E04222F0400282F0200242F41A
:1064E800004242F0800223F8212066E042F4007264
:1064F800AAE742F4C0620020A6E742F480620020C6
:10650800A2E70120A0E7097833F8212092B222F40B
:10651800E04222F0400242F4004242F0800223F8B6
:1065280021204AE0B3F8502013FA82F20C7802EBEB
:10653800C402B1F806C04FEA5C0C4FEA4C0CA2F852
:1065480004C4B3F8502013FA82F20C7802EBC402A8
:106558000C693E2C32D94FEA541C14F01F0F01D19C
:106568000CF1FF3C6FEACC6C6FEA5C4C1FFA8CFCB8
:10657800A2F806C40C7833F8242012F4804F0CD00B
:1065880033F8242092B222F4E04222F0700242F45E
:10659800404242F0800223F82420097833F8212071
:1065A80092B222F4804222F0700282F4405242F405
:1065B800004242F0800223F8212010BD8CB9B2F8C5
:1065C8000644A4B224F4F844A4B2A2F80644B2F8EB
:1065D80006446FEA44446FEA5444A4B2A2F806445D
:1065E800C8E74FEA540C14F0010F01D00CF1010C6C
:1065F8004FEA8C2C1FFA8CFCA2F806C4BAE7CA78BA
:10660800022A72D00C7833F8242092B222F4E242A3
:1066180022F0700242F4004242F0800223F8242063
:10662800B3F8502013FA82F291F800C002EBCC02C2
:10663800B1F808C04FEA5C0C4FEA4C0CA2F800C451
:10664800B3F8502013FA82F291F800C002EBCC02A2
:10665800B1F80AC04FEA5C0C4FEA4C0CA2F804C42B
:106668004A78002A50D10C7833F8242012F4804F4D
:106678000CD033F8242092B222F4E04222F07002C7
:1066880042F4404242F0800223F824200C7833F888
:10669800242012F0400F0CD033F8242092B222F4B8
:1066A800E04222F0700242F4004242F0C00223F8B5
:1066B800242091F800C033F82C2092B222F48042B2
:1066C80022F0700282F4405248F28004224323F8F8
:1066D8002C20097833F8212092B222F4E04222F0EB
:1066E8004002224323F8212067E70C7833F824205E
:1066F80092B222F4E04222F0700242F4014242F0E7
:10670800800223F824208BE70C7833F8242012F435
:10671800804F0CD033F8242092B222F4E04222F0C9
:10672800700242F4404242F0800223F824200C78A0
:1067380033F8242012F0400F0CD033F8242092B202
:1067480022F4E04222F0700242F4004242F0C00219
:1067580023F82420CA78012A1ED00C7833F8242084
:1067680092B222F4E04222F0400282F0200242F487
:10677800004242F0800223F82420097833F82120CF
:1067880092B222F4804222F0700242F4004242F0B7
:10679800800223F8212010E70C7833F8242092B2E5
:1067A80022F4E04222F0400242F4004242F0800229
:1067B80023F82420E1E70B7B002B46D14B7813B359
:1067C8000A7830F8223013F0400F0CD030F822301D
:1067D8009BB223F4E04323F0700343F4004343F0F7
:1067E800C00320F822300A7830F822309BB223F414
:1067F800E04323F0400343F4004343F0800320F8D0
:106808002230002070470A7830F8223013F4804F85
:106818000CD030F822309BB223F4E04323F070030D
:1068280043F4404343F0800320F822300A7830F8DC
:1068380022309BB223F4804323F0700343F40043D7
:1068480043F0800320F82230DBE74B78002B4ED151
:106858000A7830F8223013F4804F0CD030F8223008
:106868009BB223F4E04323F0700343F4404343F026
:10687800800320F822300A7830F8223013F0400FD5
:106888000CD030F822309BB223F4E04323F070039D
:1068980043F4004343F0C00320F822300A7830F86C
:1068A80022309BB223F4E04323F0700343F4004307
:1068B80043F0C00320F822300A7830F822309BB227
:1068C80023F4804323F0700348F2800C43EA0C035E
:1068D80020F822300A7830F822309BB223F4E043C3
:1068E80023F0400343EA0C0320F8223089E70A78B2
:1068F80030F8223013F4804F0CD030F822309BB29D
:1069080023F4E04323F0700343F4404343F080034F
:1069180020F822300A7830F8223013F0400F0CD0DB
:1069280030F822309BB223F4E04323F0700343F4A1
:10693800004343F0C00320F822300A7830F82230B0
:106948009BB223F4E04323F0700343F4404343F045
:10695800800320F822300A7830F822309BB223F4E2
:10696800E04323F0400348F2800C43EA0C0320F88C
:1069780022300A7830F822309BB223F4804323F087
:10698800700343EA0C0320F822303AE74B788BB1C6
:106998000A7830F822309BB223F4E04323F0400316
:1069A80083F0100343F4004343F0800320F82230BF
:1069B800002070470A7830F822309BB223F48043D5
:1069C80023F0700383F4805343F4004343F08003BF
:1069D80020F82230ECE70B7B002B4BD14B7833B3FC
:1069E8000A7830F8223013F0400F0CD030F82230FB
:1069F8009BB223F4E04323F0700343F4004343F0D5
:106A0800C00320F82230CB78012B33D00A7830F835
:106A180022309BB223F4E04323F0400383F02003A9
:106A280043F4004343F0800320F8223022E00A7840
:106A380030F8223013F4804F0CD030F822309BB25B
:106A480023F4E04323F0700343F4404343F080030E
:106A580020F822300A7830F822309BB223F48043A1
:106A680023F0700383F4405343F4004343F080035E
:106A780020F822300020704711B98023A0F84C304C
:106A880000207047B0F858306FEA43436FEA534329
:106A98009BB2A0F8583000207047B0F8440080B28C
:106AA800704701335B08024402F5806208E0087809
:106AB80091F801C040EA0C2022F8020B0231013B98
:106AC800002BF4D1704770B505460C464A78012A68
:106AD80032D00B7B002B40F083828B690A6993428A
:106AE80040F25D829B1A8B61B5F8503015FA83F33A
:106AF800217803EBC1033E2A40F25582510912F076
:106B08001F0F00D101396FEAC1616FEA514189B2A3
:106B1800A3F80614227835F822309BB223F4804378
:106B280023F0700383F4405343F4004343F080039D
:106B380025F82230002070BD8E6909698E4200D97F
:106B48000E46237B2BB3E378022B44D0236A9B1B8E
:106B58002362237835F8231011F0400F00F0DC8110
:106B6800002A40F0C981B5F8502015FA82F202EBEC
:106B7800C3033E2E40F2A381720916F01F0F00D105
:106B8800013A6FEAC2626FEA524292B2A3F806244F
:106B9800BBE1B6B23346E28861692846FFF781FF58
:106BA800B5F8503015FA83F3227803EBC203A3F843
:106BB8000264227835F822309BB223F4E04323F0B4
:106BC800400383F0300343F4004343F0800325F887
:106BD80022300020AFE7236A994280F05281227860
:106BE80035F822309BB223F4E04323F0700343F4DA
:106BF800014343F0800325F82230236A9B1B23625C
:106C0800237835F8232012F0400F00F09D80627839
:106C18008ABBB5F8502015FA82F202EBC3033E2E68
:106C28000CD9720916F01F0F00D1013A6FEAC2623F
:106C38006FEA524292B2A3F806241EE08EB9B3F866
:106C4800062492B222F4F84292B2A3F80624B3F8CA
:106C580006246FEA42426FEA524292B2A3F806242F
:106C68000BE0720816F0010F00D00132920292B2C6
:106C7800A3F8062401E0012A27D0B3B2628961692A
:106C88002846FFF70EFF636933446361236A22696C
:106C9800934224D99B1B23626378002B40D1B5F81B
:106CA800503015FA83F3227803EBC2033E2E1AD92B
:106CB800720916F01F0F00D1013A6FEAC2626FEA3B
:106CC800524292B2A3F802242CE0B5F8502015FAEB
:106CD80082F202EBC303B2B2A3F80624CDE7002286
:106CE80022621E46D8E78EB9B3F8022492B222F483
:106CF800F84292B2A3F80224B3F802246FEA42429F
:106D08006FEA524292B2A3F802240BE0720816F01E
:106D1800010F00D00132920292B2A3F8022401E0DE
:106D2800012B06D0B3B2228961692846FFF7B9FE64
:106D38003FE7B5F8503015FA83F3227803EBC20326
:106D4800B2B2A3F80224EDE762788ABBB5F8502006
:106D580015FA82F202EBC3033E2E0CD9720916F023
:106D68001F0F00D1013A6FEAC2626FEA524292B233
:106D7800A3F802241EE08EB9B3F8022492B222F4DA
:106D8800F84292B2A3F80224B3F802246FEA42420E
:106D98006FEA524292B2A3F802240BE0720816F08E
:106DA800010F00D00132920292B2A3F8022401E04E
:106DB800012A27D0B3B2228961692846FFF771FEFC
:106DC800636933446361236A2269934224D99B1B14
:106DD80023626378002B40D1B5F8503015FA83F35D
:106DE800227803EBC2033E2E1AD9720916F01F0F40
:106DF80000D1013A6FEAC2626FEA524292B2A3F836
:106E080006242CE0B5F8502015FA82F202EBC303F1
:106E1800B2B2A3F80224CDE7002222621E46D8E7C8
:106E28008EB9B3F8062492B222F4F84292B2A3F8CB
:106E38000624B3F806246FEA42426FEA524292B23D
:106E4800A3F806240BE0720816F0010F00D00132F7
:106E5800920292B2A3F8062401E0012B06D0B3B245
:106E6800628961692846FFF71CFEA2E6B5F8503032
:106E780015FA83F3227803EBC203B2B2A3F806240F
:106E8800EDE7217835F8212092B222F4E24222F08F
:106E9800700242F4004242F0800225F82120B5F841
:106EA800502015FA82F2217802EBC1029BB2A2F8B7
:106EB8000234228961692846FFF7F3FD79E68EB925
:106EC800B3F8062492B222F4F84292B2A3F8062448
:106ED800B3F806246FEA42426FEA524292B2A3F82C
:106EE800062412E0720816F0010F00D00132920257
:106EF80092B2A3F8062408E0B5F8502015FA82F2F9
:106F080002EBC303B2B2A3F80624B3B26289616983
:106F18002846FFF7C6FD4CE68ABBB5F8502015FA9F
:106F280082F202EBC3033E2E0CD9720916F01F0F32
:106F380000D1013A6FEAC2626FEA524292B2A3F8F4
:106F4800022425E08EB9B3F8022492B222F4F84262
:106F580092B2A3F80224B3F802246FEA42426FEA1D
:106F6800524292B2A3F8022412E0720816F0010FFE
:106F780000D00132920292B2A3F8022408E0B5F8D8
:106F8800502015FA82F202EBC303B2B2A3F802242E
:106F9800B3B2228961692846FFF783FD09E600221A
:106FA8008A611A46A0E58AB9B3F8062492B222F497
:106FB800F84292B2A3F80624B3F806246FEA4242D4
:106FC8006FEA524292B2A3F80624A3E5510812F0E0
:106FD800010F00D00131890289B2A3F8061499E59E
:106FE800CB78022B3BD0012B40F01B8189692369A8
:106FF800994240F2CA80C91AA161AAB9B5F85020CD
:1070080015FA82F2217802EBC1023E2B40F2C180D0
:10701800590913F01F0F00D101396FEAC1616FEAF6
:10702800514189B2A2F802146278002A40F0EB803C
:10703800B5F8502015FA82F2217802EBC1023E2BF6
:1070480040F2C480590913F01F0F00D101396FEACB
:10705800C1636FEA53439BB2A2F806345AE5AAB952
:10706800B0F8503010FA83F30A7803EBC2030969C9
:107078003E2925D94A0911F01F0F00D1013A6FEABC
:10708800C2626FEA524292B2A3F802246378002BDC
:1070980050D1B5F8503015FA83F3227803EBC203C8
:1070A80021693E2929D94A0911F01F0F00D1013A57
:1070B8006FEAC2626FEA524292B2A3F806243BE03A
:1070C80089B9B3F8022492B222F4F84292B2A3F832
:1070D8000224B3F802246FEA42426FEA524292B2A3
:1070E800A3F80224D2E74A0811F0010F00D00132B8
:1070F800920292B2A3F80224C8E789B9B3F8062429
:1071080092B222F4F84292B2A3F80624B3F8062405
:107118006FEA42426FEA524292B2A3F806240BE0A9
:107128004A0811F0010F00D00132920292B2A3F87E
:10713800062401E0012B1DD0E369002B3FF4EAACE3
:10714800227835F8221044F2400303EA01008B4309
:1071580002D000287FF4DEAC35F822309BB223F44D
:10716800E04323F0700343F4004343F0C00325F8E1
:107178002230CFE4B5F8503015FA83F3227803EBC8
:10718800C203228AA3F80624D6E70023A3610B468C
:1071980033E78BB9B2F8021489B221F4F84189B205
:1071A800A2F80214B2F802146FEA41416FEA5141A1
:1071B80089B2A2F8021437E7590813F0010F00D07A
:1071C8000131890289B2A2F802142DE78BB9B2F80D
:1071D80006349BB223F4F8439BB2A2F80634B2F803
:1071E80006346FEA43436FEA53439BB2A2F806346E
:1071F80090E4590813F0010F00D001318B029BB2C3
:10720800A2F8063486E4012A7FF484ACB5F850204D
:1072180015FA82F2217802EBC1029BB2A2F8063479
:1072280078E4012087E410B45C08024402F5806227
:1072380007E032F8020B0870C0F3072048700231EB
:10724800013C002CF5D113F0010F01D013880B700D
:107258005DF8044B704798B108B503460020C3F8A1
:10726800B802C3F8C002C3F8CC0209B1C3F8B4121B
:10727800012183F89C121A701846FDF749FF08BDD2
:107288000320704710B582B00023ADF8063061B115
:107298000446C0F8B812CB6A4BB10DF10600984706
:1072A800C4F8CC02002002B010BD0320FBE7002088
:1072B800F9E708B5FDF762FF08BD08B5D0F8B832A0
:1072C80013B11B68984708BD0320FCE708B5D0F840
:1072D800B8320BB15B689847002008BD38B5044642
:1072E80000F2AA25284600F02FF90123C4F89432A9
:1072F800B4F8B032C4F8983294F8AA1201F01F0317
:10730800012B0DD0022B10D02BB101F080012046AB
:10731800FDF74FFF03E02946204600F0E4FA38BDA8
:107328002946204600F017FBF9E72946204600F0D9
:1073380046FBF4E738B504460D4641BB1346D0F882
:107348009422032A01D0084638BDD0F85C11D0F841
:107358006021914209D890F89C32DBB2032B0FD000
:10736800204600F06BFC2846EEE7891AC0F85C114D
:107378008A4228BF0A46194600F058FC2846E3E727
:10738800D0F8B8321B69002BEAD09847E8E790F8A4
:107398009C32DBB2032B01D00020D5E7D0F8B832FD
:1073A8009B690BB19847CFE70020CDE738B5044675
:1073B8000D4600294AD11346D0F89422022A05D056
:1073C80094F8A032012B3CD0284638BDC269016A26
:1073D8008A420ED88A4218D094F89C32DBB2032B2A
:1073E80027D080212046FDF7E4FE204600F031FC3E
:1073F800E6E7521AC261194600F001FC00231A465A
:1074080019462046FDF70CFFDAE783699942E3D86D
:10741800D0F898229342DFD20022114600F0EFFB09
:107428000021C4F898120B460A462046FDF7F8FEDC
:10743800C6E7D4F8B832DB68002BD2D0204698478C
:10744800CFE7002384F8A0322846BEE790F89C32A4
:10745800DBB2032B01D00020B7E7D0F8B8325B6964
:107468000BB19847B1E70020AFE7012380F89C32C1
:107478000023C0F894324360C0F8A432D0F8B83280
:10748800F3B170B50446D0F8BC221AB15B680BB1F1
:10749800002198474023002211462046FDF776FE3A
:1074A8000126A4F864614025C4F860512B460022E7
:1074B80080212046FDF76AFEA6842562002070BD63
:1074C8000320704701740020704790F89C32DBB2AB
:1074D80080F89D32042380F89C320020704790F891
:1074E8009C32DBB2042B01D00020704790F89D320B
:1074F800DBB280F89C32F7E7D0F8B82262B108B561
:1075080090F89C32DBB2032B01D0002008BDD36970
:1075180023B198470020F9E7032070470020F5E7DA
:107528000346002002E00130C0B201331A78002A75
:10753800F9D1704708B54B88012B00D008BDC0F8B9
:10754800A43200F07BFBF9E70B7803704B784370AB
:107558008B78CA7843EA022343800B794A7943EA55
:10756800022383808B79CA7943EA0223C380704758
:1075780010B504468021FDF71CFE00212046FDF7CA
:1075880018FE10BD30B583B004460D460023ADF893
:1075980006304A88130A013B0E2B00F2BC80DFE854
:1075A80003F0153044BABA9EABBABABABABABABA84
:1075B8000800D0F8B432DB6923B10DF10601007C74
:1075C80098470AE02946FFF7D3FF18E0D0F8B4320D
:1075D8001B680DF10601007C9847EA88002A00F034
:1075E800A380BDF80630002B00F099809A4228BF8E
:1075F8001A46ADF806200146204600F0F3FA03B01B
:1076080030BD037C43B9D0F8B8329B6A0DF106004F
:10761800984702234370E0E7D0F8B832DB6A0DF1EF
:107628000600984702234370D7E7D2B2052A52D8FA
:10763800DFE802F003101D2A3744D0F8B4325B6843
:1076480023B10DF10601007C9847C6E72946FFF7EC
:107658008FFFD4E7D0F8B4329B6823B10DF106014F
:10766800007C9847B9E72946FFF782FFC7E7D0F8BB
:10767800B432DB6823B10DF10601007C9847ACE712
:107688002946FFF775FFBAE7D0F8B4321B6923B172
:107698000DF10601007C98479FE72946FFF768FF30
:1076A800ADE7D0F8B4325B6923B10DF10601007C77
:1076B800984792E72946FFF75BFFA0E7D0F8B43276
:1076C8009B6923B10DF10601007C984785E729469F
:1076D800FFF74EFF93E72946FFF74AFF8FE7037C42
:1076E80033B9D0F8B8325B6B0DF10600984774E7F0
:1076F8002946FFF73DFF82E7037C43B9D0F8B8324B
:107708001B6B0DF1060098470723437065E7294670
:10771800FFF72EFF73E72946FFF72AFF6FE7294691
:107728002046FFF725FF6AE7204600F087FA66E75C
:1077380038B504468B88FBB9CB88EBB94B887F2BCF
:107748001AD803F07F0590F89C32DBB2032B0CD0DB
:1077580080F89E522946FDF753FD204600F06EFA48
:1077680035B1022384F89C3209E0FFF701FF06E0F7
:10777800012384F89C3202E02046FFF7F9FE38BD69
:1077880070B504460E468D782E4B1D70012D10D80D
:1077980090F89C32DBB2022B0FD0032B23D0FFF7DB
:1077A800E7FE284B19782046FFF790FD0325284669
:1077B80070BDFFF7DDFE0325F9E78DB14560294669
:1077C800FFF77BFD054620B131462046FFF7D0FE86
:1077D800EDE7204600F032FA032384F89C32E6E70E
:1077E80000F02CFAE3E7CDB141688D4225D0C9B24B
:1077F800FFF76CFD134B197861602046FFF75DFDBC
:107808000546B0B131462046FFF7B2FE2179204641
:10781800FFF75CFD022384F89C32C8E7022380F856
:107828009C3245602946FFF751FD204600F006FAD4
:10783800BDE7204600F002FAB9E700F0FFF900259D
:10784800B5E700BF3C27002008B5CB88012B0BD13A
:1078580090F89C32DBB2022B09D9032B09D1012203
:10786800011D00F0BFF901E0FFF782FE08BD5BB221
:1078780013B9FFF77DFEF9E70146002341F8083FF9
:10788800012200F0AFF9F1E708B590F89C32013B0E
:10789800022B12D8CB88022B0CD10123C360D0F85D
:1078A800A4320BB10323C360022200F10C0100F0E3
:1078B80099F908BDFFF75CFEFBE7FFF759FEF8E70B
:1078C80008B590F89C32013B022B09D84B88012B54
:1078D80000D008BD0023C0F8A43200F0AFF9F8E7E3
:1078E800FFF746FEF5E738B50C7804F06004202C65
:1078F80006D0402C04D054B1FFF73AFE002404E02F
:10790800D0F8B8329B6898470446204638BD4D7871
:10791800092D1DD8DFE805F012191C161C08051CD6
:107928000F0BFFF72FFEF0E7FFF702FFEDE7FFF77A
:1079380027FF0446E9E7FFF787FFE6E7FFF7A4FF1D
:107948002C46E2E7FFF7F6FDDFE7FFF7B9FFDCE7D4
:10795800FFF70EFED9E770B505460C460B7803F025
:107968006003202B07D0402B05D023B1FFF700FE82
:107978000026304670BD95F89C32013B022B18D882
:107988002379012B0FD8D5F8B8329B6821462846B1
:1079980098470646E388002BEBD10028E9D1284612
:1079A80000F04CF9E5E721462846FFF7E1FD0026FF
:1079B800DFE721462846FFF7DBFD0026D9E7F8B5C3
:1079C80006460D468B880C7804F06004202C08D0FD
:1079D800D9B2402C05D06CB12946FFF7C9FD002467
:1079E80006E0D6F8B8329B682946304698470446E0
:1079F8002046F8BD6F78012F2FD0032F05D0002F18
:107A080059D02946FFF7B4FDF2E790F89C32DBB273
:107A1800022B05D0032B12D02946FFF7A9FDE7E773
:107A280009B1802904D129463046FFF7A1FDDFE7D7
:107A3800FDF7BFFB80213046FDF7BBFBD8E76B881D
:107A480023B919B1802901D0EB881BB1304600F069
:107A5800F5F8CDE7FDF7ADFBF8E790F89C32DBB21F
:107A6800022B05D0032B12D02946FFF781FDBFE773
:107A780009B1802904D129463046FFF779FDB7E7D7
:107A8800FDF797FB80213046FDF793FBB0E76B8845
:107A9800002BADD111F07F0F0AD1304600F0CEF89F
:107AA800D6F8B8329B6829463046984704469FE77F
:107AB800FDF787FBF1E790F89C22D2B2022A06D0A4
:107AC800032A29D02946FFF753FD3C4690E709B120
:107AD800802913D113F0800F15D101F07F0101EB3C
:107AE8008101890001F5A8713144043100230B603C
:107AF8000222304600F076F83C4679E72946FFF73F
:107B080037FD3C4674E701F07F0101EB81018900F4
:107B1800103131440431E9E75BB2002B1FDB01F07F
:107B28000F0202EB820200EB8202B2F8642122B358
:107B3800002B27DB01F07F0303EB83039C0004F594
:107B4800A8743444043409B1802924D10023236063
:107B580002222146304600F045F83C4648E701F04D
:107B68000F0202EB820200EB8202928C002ADFD124
:107B78002946FFF7FDFC3C463AE72946FFF7F8FCA3
:107B88003C4635E701F07F0303EB83039C00103488
:107B980034440434D7E73046FDF71BFB10B101230A
:107BA8002360D5E700232360D2E7D0B170B50D4636
:107BB80016460446FFF7B4FC431C5B009BB23380B7
:107BC8002B7003236B70022307E0EA5401345A1C1C
:107BD800D2B20021A9540233DBB22278002AF4D1B0
:107BE80070BD704708B513460222C0F8942283611D
:107BF800C3610A460021FDF70BFB002008BD08B54C
:107C080013460A460021FDF703FB002008BD08B50E
:107C180013460322C0F89422C0F85831C0F85C31EA
:107C28000A460021FDF7FCFA002008BD08B51346F6
:107C38000A460021FDF7F4FA002008BD08B5042221
:107C4800C0F8942200231A461946FDF7E1FA0020ED
:107C580008BD08B50522C0F8942200231A46194623
:107C6800FDF7DEFA002008BD6D2303800048704749
:107C7800880000200020704710B5D0F8BC42ECB155
:107C880004F5805292F88A2B012A01D0002010BDF9
:107C980004F5805292F8CC2B022A01D00020F6E796
:107CA800D0F8C022126904F5805494F88B0B9047E1
:107CB800002084F88A0B84F8CB0BE8E70320E6E77A
:107CC8000020704700207047002070470020704750
:107CD8000A230380004870477C000020F8B5D0F8DC
:107CE800BC52002D4ED00446012901D00020F8BD19
:107CF800FDF79EFA86B2D4F8C0325B6905F5805765
:107D0800B7F8880B28440122314604309847B7F861
:107D1800883B33449BB2A7F8883BB3F5DC5F18D0A7
:107D280005F5805393F8853B33B905F58053B3F8CF
:107D3800883BB3F55C6F1FD005F58053B3F8883BDB
:107D4800EA185823043201212046FDF769FA002079
:107D5800CDE70022A7F8882B97F8843B032BDFD1C7
:107D6800D4F8C0329B6801224FF45C61281D984703
:107D7800002287F8842BD3E705F58053012283F886
:107D8800852BD9E70320B2E770B5D0F8BC4274B1AF
:107D980005460E4604F5DC540B34402200212046EB
:107DA800F8F77EFAF28821462846FFF71BFF70BDD8
:107DB80038B5D0F8BC5215B10C46CA8802B938BDDE
:107DC80005F5DC510B31FFF722FF05F5805501233E
:107DD80085F88A3BA37985F8CB3BA3881B0A85F8ED
:107DE800CC3BECE730B583B00023ADF80630D0F8D3
:107DF800BC32002B67D00C7814F0600412D0202C11
:107E08005BD14B78012B05D0812B07D1FFF7BCFF45
:107E1800002455E0FFF7CCFF002451E0FFF7A8FB52
:107E280003244DE04D780B2D43D8DFE805F00649D3
:107E38004242424216424242223090F89C32DBB221
:107E4800032B03D0FFF794FB032439E002220DF142
:107E58000601FFF7C7FE2C4632E04B881B0A212B90
:107E68002ED1CA88092A28BF09221849FFF7BAFE65
:107E780026E090F89C22D2B2032A03D0FFF778FBC1
:107E880003241DE001221946FFF7ACFE18E090F824
:107E98009C52EDB2032D08D18A78012A01D81A60C4
:107EA8000EE0FFF765FB2C460AE0FFF761FB0324B1
:107EB80006E0FFF75DFB032402E0FFF759FB03240C
:107EC800204603B030BD0324FAE700BF9A00002023
:107ED80010B504460121FDF764F90023A4F87831B0
:107EE800A4F87A31D4F8BC325BB1D4F8C0325B68FC
:107EF80000209847D4F8BC02FDF7C8F90023C4F85D
:107F0800BC32002010BD38B5044641F6D030FDF72C
:107F1800B9F968B30546C4F8BC02237C6BBB0123DE
:107F2800A4F87A315823012211462046FDF72EF98C
:107F38000123A4F8783100222A6005F58053032133
:107F480083F8841BA3F8882BA3F8862B83F8852B4A
:107F5800D4F8C0321B68462145F25460984780B96E
:107F680058232A1D01212046FDF75AF9002038BD63
:107F78000023C4F8BC320220F9E70123A4F87A31BF
:107F8800D0E70320F3E719B1C0F8C012002070470A
:107F9800032070470D4885460D480E490E4A0023B8
:107FA80002E0D458C4500433C4188C42F9D30B4AA5
:107FB8000B4C002301E013600432A242FBD3FCF710
:107FC800D9FFF8F749F9F9F77FF9FEE700800020B3
:107FD8000000002030010020A080000830010020AF
:107FE80040270020FEE70000F8B500BFF8BC08BC39
:107FF8009E467047F8B500BFF8BC08BC9E4670475F
:10800800010002000400060008000A000C0010002D
:10801800200040008000000108040204080101015A
:108028000101010307010000000000000102030430
:108038000000000000000000010203040607080910
:1080480053544D333220417564696F20436C61731A
:108058007300000053544D6963726F656C656374F7
:10806800726F6E6963730000415544494F20436F36
:108078006E66696700000000415544494F20496E0B
:08808800746572666163650016
:08809000188BFF7F01000000C6
:048098004102000899
:04809C0019020008BD
:1080A00001000000100000000024F4001A0300008A
:1080B00000000000000000000000000000000000C0
:1080C0000000000000000000040309041201000287
:1080D0000000004083044057000201020301000039
:1080E00099520008A552000869530008455300083A
:1080F0003153000885530008A95300080000000010
:10810000CD530008D1530008D5530008D9530008B7
:10811000DD530008E1530008E55300080A06000299
:10812000000000400100000009026D00020100C0D3
:1081300032090400000001010000092401000127A8
:108140000001010C240201010100010000000009EE
:1081500024060201010100000924030301030002B7
:1081600000090401000001020000090401010101ED
:10817000020000072401010101000B240201020298
:10818000100154560009050101580001000007259F
:1081900001000000000000000F7F0008D97E0008E9
:1081A000ED7D0008C97C0008817C00087D7C00080A
:1081B000E57C0008CD7C0008D17C0008D57C000857
:1081C000717C0008717C0008717C0008D97C000873
:0400000508007F9DD3
:00000001FF
